:020000040800F2
:1040000000000120A5950008898A00088B8A000815
:104010008D8A00088F8A0008918A0008000000003D
:10402000000000000000000000000000938A00086B
:10403000958A000800000000978A0008998A000805
:10404000ED950008ED950008ED950008ED95000848
:10405000ED950008ED950008ED950008ED95000838
:10406000ED950008ED950008ED9500089D8A000883
:10407000ED950008ED950008A98A0008B58A0008AA
:10408000ED950008ED950008ED950008ED95000808
:10409000ED950008ED950008ED950008ED950008F8
:1040A000ED950008ED950008ED950008ED950008E8
:1040B000ED950008ED950008ED950008ED950008D8
:1040C000ED950008ED950008ED950008ED950008C8
:1040D000ED950008C18A0008ED950008ED950008EF
:1040E000ED950008ED950008ED950008ED950008A8
:1040F000ED950008ED950008ED950008ED95000898
:10410000ED950008ED950008ED950008ED95000887
:10411000ED950008ED950008CD8A0008ED950008A2
:10412000ED950008ED950008ED950008ED95000867
:10413000000000000000000000000000000000007F
:10414000000000000000000000000000000000006F
:10415000000000000000000000000000000000005F
:10416000000000000000000000000000000000004F
:10417000000000000000000000000000000000003F
:10418000000000000000000000000000000000002F
:10419000000000000000000000000000000000001F
:1041A000000000000000000000000000000000000F
:1041B00000000000000000000000000000000000FF
:1041C00000000000000000000000000000000000EF
:1041D00000000000000000000000000000000000DF
:0441E0005FF8E0F1B3
:1041E80010B5054C237833B9044B13B10448AFF329
:1041F80000800123237010BD080400200000000087
:1042080024BF000808B5034B1BB103490348AFF3AB
:10421800008008BD000000000C04002024BF000836
:10422800034613F8012B002AFBD1181A01387047EE
:10423800D0400B1CD1409C46203AD34018435242F0
:10424800634693401843704781F0004102E000BF85
:1042580083F0004330B54FEA41044FEA430594EA3E
:10426800050F08BF90EA020F1FBF54EA000C55EA79
:10427800020C7FEA645C7FEA655C00F0E2804FEA4A
:104288005454D4EB5555B8BF6D420CDD2C4480EA2C
:10429800020281EA030382EA000083EA010180EA5C
:1042A800020281EA0303362D88BF30BD11F0004FAA
:1042B8004FEA01314FF4801C4CEA113102D04042E0
:1042C80061EB410113F0004F4FEA03334CEA13331B
:1042D80002D0524263EB430394EA050F00F0A78033
:1042E800A4F10104D5F1200E0DDB02FA0EFC22FA2E
:1042F80005F2801841F1000103FA0EF2801843FA22
:1043080005F359410EE0A5F120050EF1200E012A12
:1043180003FA0EFC28BF4CF0020C43FA05F3C01850
:1043280051EBE37101F0004507D54FF0000EDCF1C9
:10433800000C7EEB00006EEB0101B1F5801F1BD372
:10434800B1F5001F0CD349085FEA30004FEA3C0C76
:1043580004F101044FEA445212F5800F80F09A806C
:10436800BCF1004F08BF5FEA500C50F1000041EB70
:10437800045141EA050130BD5FEA4C0C404141EB74
:10438800010111F4801FA4F10104E9D191F0000F9B
:1043980004BF01460020B1FA81F308BF2033A3F11E
:1043A8000B03B3F120020CDA0C3208DD02F1140C15
:1043B800C2F10C0201FA0CF021FA02F10CE002F150
:1043C8001402D8BFC2F1200C01FA02F120FA0CFC49
:1043D800DCBF41EA0C019040E41AA2BF01EB045192
:1043E800294330BD6FEA04041F3C1CDA0C340EDC90
:1043F80004F11404C4F1200220FA04F001FA02F3D3
:1044080040EA030021FA04F345EA030130BDC4F190
:104418000C04C4F1200220FA02F001FA04F340EA85
:104428000300294630BD21FA04F0294630BD94F036
:10443800000F83F4801306BF81F480110134013D1D
:104448004EE77FEA645C18BF7FEA655C29D094EA8E
:10445800050F08BF90EA020F05D054EA000C04BF0C
:104468001946104630BD91EA030F1EBF00210020F7
:1044780030BD5FEA545C05D14000494128BF41F096
:10448800004130BD14F580043CBF01F5801130BDFA
:1044980001F0004545F0FE4141F470014FF0000085
:1044A80030BD7FEA645C1ABF194610467FEA655C36
:1044B8001CBF0B46024650EA013406BF52EA0335D8
:1044C80091EA030F41F4002130BD00BF90F0000FC6
:1044D80004BF0021704730B54FF4806404F1320402
:1044E8004FF000054FF0000150E700BF90F0000FBB
:1044F80004BF0021704730B54FF4806404F13204E2
:1045080010F0004548BF40424FF000013EE700BFB1
:1045180042004FEAE2014FEA31014FEA02701FBF41
:1045280012F07F4393F07F4F81F06051704792F013
:10453800000F14BF93F07F4F704730B54FF460748D
:1045480001F0004521F0004120E700BF50EA0102D8
:1045580008BF704730B54FF000050AE050EA010285
:1045680008BF704730B511F0004502D5404261EBF5
:1045780041014FF4806404F132045FEA915C3FF436
:10458800DCAE4FF003025FEADC0C18BF03325FEACF
:10459800DC0C18BF033202EBDC02C2F1200300FA84
:1045A80003FC20FA02F001FA03FE40EA0E0021FAA9
:1045B80002F11444C1E600BF70B54FF0FF0C4CF493
:1045C800E06C1CEA11541DBF1CEA135594EA0C0F49
:1045D80095EA0C0F00F0DEF82C4481EA030621EA84
:1045E8004C5123EA4C5350EA013518BF52EA0335BF
:1045F80041F4801143F4801338D0A0FB02CE4FF071
:104608000005E1FB02E506F00042E0FB03E54FF0A0
:104618000006E1FB03569CF0000F18BF4EF0010E98
:10462800A4F1FF04B6F5007F64F5407404D25FEA94
:104638004E0E6D4146EB060642EAC62141EA555147
:104648004FEAC52040EA5E504FEACE2EB4F1FD0C89
:1046580088BFBCF5E06F1ED8BEF1004F08BF5FEA07
:10466800500E50F1000041EB045170BD06F00046B9
:1046780046EA010140EA020081EA0301B4EB5C0466
:10468800C2BFD4EB0C0541EA045170BD41F480115E
:104698004FF0000E013C00F3AB8014F1360FDEBF83
:1046A800002001F0004170BDC4F10004203C35DA5F
:1046B8000C341BDC04F11404C4F1200500FA05F3E2
:1046C80020FA04F001FA05F240EA020001F0004283
:1046D80021F0004110EBD37021FA04F642EB0601F9
:1046E8005EEA430E08BF20EAD37070BDC4F10C0423
:1046F800C4F1200500FA04F320FA05F001FA04F2E7
:1047080040EA020001F0004110EBD37041F10001D2
:104718005EEA430E08BF20EAD37070BDC4F12005DD
:1047280000FA05F24EEA020E20FA04F301FA05F245
:1047380043EA020321FA04F001F0004121FA04F2ED
:1047480020EA020000EBD3705EEA430E08BF20EABD
:10475800D37070BD94F0000F0FD101F000464000F7
:1047680041EB010111F4801F08BF013CF7D041EA79
:10477800060195F0000F18BF704703F0004652007D
:1047880043EB030313F4801F08BF013DF7D043EA4E
:104798000603704794EA0C0F0CEA135518BF95EA04
:1047A8000C0F0CD050EA410618BF52EA4306D1D18B
:1047B80081EA030101F000414FF0000070BD50EAAA
:1047C800410606BF1046194652EA430619D094EA34
:1047D8000C0F02D150EA013613D195EA0C0F05D11E
:1047E80052EA03361CBF104619460AD181EA030172
:1047F80001F0004141F0FE4141F470014FF000002A
:1048080070BD41F0FE4141F4780170BD70B54FF0C4
:10481800FF0C4CF4E06C1CEA11541DBF1CEA135544
:1048280094EA0C0F95EA0C0F00F0A7F8A4EB050426
:1048380081EA030E52EA03354FEA013100F088801D
:104848004FEA03334FF0805545EA131343EA1263E6
:104858004FEA022245EA111545EA10654FEA00269B
:104868000EF000419D4208BF964244F1FD0404F554
:10487800407402D25B084FEA3202B61A65EB0305B0
:104888005B084FEA32024FF480104FF4002CB6EB6D
:10489800020E75EB030E22BFB61A754640EA0C00ED
:1048A8005B084FEA3202B6EB020E75EB030E22BF2D
:1048B800B61A754640EA5C005B084FEA3202B6EB6E
:1048C800020E75EB030E22BFB61A754640EA9C002D
:1048D8005B084FEA3202B6EB020E75EB030E22BFFD
:1048E800B61A754640EADC0055EA060E18D04FEABB
:1048F800051545EA16754FEA06164FEAC30343EA5B
:1049080052734FEAC2025FEA1C1CC0D111F4801F27
:104918000BD141EA00014FF000004FF0004CB6E720
:1049280011F4801F04BF01430020B4F1FD0C88BFBF
:10493800BCF5E06F3FF6AFAEB5EB030C04BFB6EBCA
:10494800020C5FEA500C50F1000041EB045170BDBD
:104958000EF0004E4EEA113114EB5C04C2BFD4EBEA
:104968000C0541EA045170BD41F480114FF0000E6E
:10497800013C90E645EA060E8DE60CEA135594EAEA
:104988000C0F08BF95EA0C0F3FF43BAF94EA0C0FED
:104998000AD150EA01347FF434AF95EA0C0F7FF462
:1049A80025AF104619462CE795EA0C0F06D152EAB6
:1049B80003353FF4FDAE1046194622E750EA41069A
:1049C80018BF52EA43067FF4C5AE50EA41047FF4AB
:1049D8000DAF52EA43057FF4EBAE12E74FF0FF3C10
:1049E80006E000BF4FF0010C02E000BF4FF0010CE1
:1049F8004DF804CD4FEA410C7FEA6C5C4FEA430C5A
:104A080018BF7FEA6C5C1BD001B050EA410C0CBFA8
:104A180052EA430C91EA030F02BF90EA020F00200A
:104A2800704710F1000F91EA030F58BF994208BF71
:104A380090422CBFD8176FEAE37040F0010070472E
:104A48004FEA410C7FEA6C5C02D150EA013C07D185
:104A58004FEA430C7FEA6C5CD6D152EA033CD3D0D0
:104A68005DF8040B704700BF8446104662468C46CA
:104A78001946634600E000BF01B5FFF7B7FF0028FD
:104A880048BF10F1000F01BD4DF808EDFFF7F4FF26
:104A98000CBF012000205DF808FB00BF4DF808EDB1
:104AA800FFF7EAFF34BF012000205DF808FB00BFD4
:104AB8004DF808EDFFF7E0FF94BF012000205DF8F6
:104AC80008FB00BF4DF808EDFFF7CEFF94BF0120AB
:104AD80000205DF808FB00BF4DF808EDFFF7C4FFA4
:104AE80034BF012000205DF808FB00BF4FEA410CED
:104AF8007FEA6C5C02D150EA013C0AD14FEA430CD0
:104B08007FEA6C5C02D152EA033C02D14FF000000C
:104B180070474FF0010070474FEA410212F500124A
:104B280015D211D56FF47873B3EB625212D94FEAEC
:104B3800C12343F0004343EA505311F0004F23FAD6
:104B480002F018BF404270474FF00000704750EA2B
:104B5800013005D111F0004008BF6FF000407047E8
:104B68004FF00000704700BF4A0011D212F5001242
:104B780011D20DD56FF47873B3EB62520ED44FEAAD
:104B8800C12343F0004343EA505323FA02F070472D
:104B98004FF00000704750EA013002D14FF0FF306B
:104BA80070474FF0000070474FEA4102B2F1E0430E
:104BB80024BFB3F5001CDCF1FE5C0DD901F0004CFC
:104BC8004FEAC0024CEA5070B2F1004F40EB83004C
:104BD80008BF20F00100704711F0804F21D113F178
:104BE8003872BCBF01F00040704741F480114FEAB1
:104BF8005252C2F11802C2F1200C10FA0CF320FA3A
:104C080002F018BF40F001004FEAC1234FEAD32356
:104C180003FA0CFC40EA0C0023FA02F34FEA4303C0
:104C2800CCE77FEA625307D150EA01331EBF4FF049
:104C3800FE4040F44000704701F0004040F0FE4064
:104C480040F40000704700BF80F0004002E000BF61
:104C580081F0004142001FBF5FEA410392EA030F5F
:104C68007FEA226C7FEA236C6AD04FEA1262D2EBA9
:104C78001363C1BFD218414048404140B8BF5B42AE
:104C8800192B88BF704710F0004F40F4000020F047
:104C98007F4018BF404211F0004F41F4000121F05D
:104CA8007F4118BF494292EA030F3FD0A2F10102A7
:104CB80041FA03FC10EB0C00C3F1200301FA03F1E5
:104CC80000F0004302D5494260EB4000B0F5000F08
:104CD80013D3B0F1807F06D340084FEA310102F1C7
:104CE8000102FE2A51D2B1F1004F40EBC25008BF79
:104CF80020F0010040EA03007047490040EB000043
:104D080010F4000FA2F10102EDD1B0FA80FCACF171
:104D1800080CB2EB0C0200FA0CF0AABF00EBC25070
:104D280052421843BCBFD0401843704792F0000F5E
:104D380081F4000106BF80F400000132013BB5E7B1
:104D48004FEA41037FEA226C18BF7FEA236C21D027
:104D580092EA030F04D092F0000F08BF084670478C
:104D680090EA010F1CBF0020704712F07F4F04D15A
:104D7800400028BF40F00040704712F100723CBF6D
:104D880000F50000704700F0004343F0FE4040F497
:104D9800000070477FEA226216BF08467FEA236355
:104DA8000146420206BF5FEA412390EA010F40F440
:104DB800800070474FF0000304E000BF10F000438C
:104DC80048BF40425FEA000C08BF704743F0964373
:104DD80001464FF000001CE050EA010208BF70478E
:104DE8004FF000030AE000BF50EA010208BF704715
:104DF80011F0004302D5404261EB41015FEA010C2A
:104E080002BF84460146002043F0B64308BFA3F121
:104E18008053A3F50003BCFA8CF2083AA3EBC25303
:104E280010DB01FA02FC634400FA02FCC2F1200222
:104E3800BCF1004F20FA02F243EB020008BF20F059
:104E48000100704702F1200201FA02FCC2F12002BF
:104E580050EA4C0021FA02F243EB020008BF20EAB4
:104E6800DC7070474FF0FF0C1CEAD0521EBF1CEAE2
:104E7800D15392EA0C0F93EA0C0F6FD01A4480EAD0
:104E8800010C400218BF5FEA41211ED04FF00063B9
:104E980043EA501043EA5111A0FB01310CF00040E5
:104EA800B1F5000F3EBF490041EAD3715B0040EA0B
:104EB800010062F17F02FD2A1DD8B3F1004F40EBDB
:104EC800C25008BF20F00100704790F0000F0CF0AE
:104ED800004C08BF49024CEA502040EA51207F3A72
:104EE800C2BFD2F1FF0340EAC250704740F400004D
:104EF8004FF00003013A5DDC12F1190FDCBF00F03E
:104F080000407047C2F10002410021FA02F1C2F1EB
:104F1800200200FA02FC5FEA310040F1000053EA87
:104F28004C0308BF20EADC70704792F0000F00F0D5
:104F3800004C02BF400010F4000F013AF9D040EADB
:104F48000C0093F0000F01F0004C02BF490011F46F
:104F5800000F013BF9D041EA0C018FE70CEAD1536D
:104F680092EA0C0F18BF93EA0C0F0AD030F0004CED
:104F780018BF31F0004CD8D180EA010000F00040A1
:104F8800704790F0000F17BF90F0004F084691F05F
:104F9800000F91F0004F14D092EA0C0F01D1420299
:104FA8000FD193EA0C0F03D14B0218BF084608D162
:104FB80080EA010000F0004040F0FE4040F40000AC
:104FC800704740F0FE4040F4400070474FF0FF0C3F
:104FD8001CEAD0521EBF1CEAD15392EA0C0F93EA86
:104FE8000C0F69D0A2EB030280EA010C49024FEAD8
:104FF800402037D04FF0805343EA111143EA101391
:105008000CF000408B4238BF5B0042F17D024FF448
:10501800000C8B4224BF5B1A40EA0C00B3EB510F23
:1050280024BFA3EB510340EA5C00B3EB910F24BF0C
:10503800A3EB910340EA9C00B3EBD10F24BFA3EB91
:10504800D10340EADC001B0118BF5FEA1C1CE0D159
:10505800FD2A3FF650AF8B4240EBC25008BF20F00C
:10506800010070470CF0004C4CEA50207F32C2BF60
:10507800D2F1FF0340EAC250704740F400004FF0FD
:105088000003013A37E792F0000F00F0004C02BF2E
:10509800400010F4000F013AF9D040EA0C0093F0F8
:1050A800000F01F0004C02BF490011F4000F013B52
:1050B800F9D041EA0C0195E70CEAD15392EA0C0FBA
:1050C80008D142027FF47DAF93EA0C0F7FF470AFF2
:1050D800084676E793EA0C0F04D14B023FF44CAF35
:1050E80008466EE730F0004C18BF31F0004CCAD1CA
:1050F80030F000427FF45CAF31F000437FF43CAF06
:105108005FE700BF42000ED2B2F1FE4F0BD34FF063
:105118009E03B3EB126209D44FEA002343F0004325
:1051280023FA02F070474FF00000704712F1610F48
:1051380001D1420202D14FF0FF3070474FF000001A
:10514800704700BF53B94AB9002908BF00281CBFDF
:105158004FF0FF314FF0FF3000F07AB9ADF1080C95
:105168006DE904CE00F006F8DDF804E0DDE902237D
:1051780004B070472DE9F0478C460E460446089D5A
:10518800002B50D18A4217466CD9B2FA82FEBEF182
:10519800000F0BD0CEF1200C01FA0EF620FA0CFC11
:1051A80002FA0EF74CEA060C00FA0EF43A0CBCFBB5
:1051B800F2F9BBB202FB19CC09FB03FA4FEA144817
:1051C80048EA0C46B2450AD9F61909F1FF3180F0D0
:1051D8002581B24540F22281A9F102093E44A6EB9D
:1051E8000A06B6FBF2F002FB106600FB03F3A4B25A
:1051F80044EA0644A34209D9E41900F1FF3280F0D9
:105208000B81A34240F2088102383C440021E41A91
:1052180040EA0940002D62D0002324FA0EF42C60E5
:105228006B60BDE8F0878B4207D9002D55D000216F
:1052380085E841000846BDE8F087B3FA83F1002904
:1052480040F08F80B34202D3824200F2FC80841A7D
:1052580066EB03060120B446002D40D085E8101007
:10526800BDE8F08712B90127B7FBF2F7B7FA87FE56
:10527800BEF1000F35D10121F61B4FEA174C1FFA7A
:1052880087F8B6FBFCF20CFB126608FB02F0230C55
:1052980043EA0646B04207D9F61902F1FF3302D2B3
:1052A800B04200F2D2801A46361AB6FBFCF00CFB6C
:1052B800106608FB00F8A3B243EA0644A04507D9E4
:1052C800E41900F1FF3302D2A04500F2B980184674
:1052D800A4EB080440EA02409CE729462846BDE8BA
:1052E800F08707FA0EF7CEF1200326FA03F24FEA09
:1052F800174CB2FBFCF11FFA87F80CFB112206FAD7
:105308000EF620FA03F301FB08F933431E0C46EAB4
:105318000246B14500FA0EF409D9F61901F1FF3237
:1053280080F08C80B14540F2898002393E44A6EB7A
:105338000906B6FBFCF00CFB106200FB08F99EB2F4
:1053480046EA0246B14507D9F61900F1FF3371D292
:10535800B1456FD902383E44A6EB090640EA01413F
:105368008FE7C1F1200722FA07F88B4048EA0303C8
:1053780026FA07F44FEA134EB4FBFEF91FFA83FC32
:105388000EFB19448E4020FA07F809FB0CFA48EA8C
:1053980006084FEA184646EA0444A24502FA01F212
:1053A80000FA01F608D9E41809F1FF3044D2A24501
:1053B80042D9A9F102091C44A4EB0A04B4FBFEF08B
:1053C8000EFB104400FB0CFC1FFA88F848EA044462
:1053D800A44507D9E41800F1FF3E29D2A44527D9EE
:1053E80002381C4440EA0940A0FB0289A4EB0C0CDB
:1053F800CC45C246CE4615D312D055B1B6EB0A03FA
:105408006CEB0E0606FA07F7CB401F43CE402F6021
:105418006E600021BDE8F0871046F7E68946DEE6B3
:105428004645EAD2B8EB020A69EB030E0138E4E715
:105438007046D7E718468FE78146BDE7114676E7FD
:1054480002383C4444E7084606E7023A3E442BE764
:10545800704700BF38B50E4B054618784FF47A737D
:10546800B3FBF0F30B4A1068B0FBF3F000F038FB25
:10547800044658B90F2D09D8024629464FF0FF3087
:1054880000F0EEFA044B20461D6038BD012038BDFF
:10549800000000200002002004000020074A08B590
:1054A8001368032043F01003136000F0C7FA0020CC
:1054B800FFF7D0FF03F0D2F9002008BD002002401A
:1054C800034A044B11681B780B441360704700BFF4
:1054D8005C04002000000020014B1868704700BFE2
:1054E8005C04002038B50446FFF7F6FF0546631C48
:1054F8001EBF044B1B78E418FFF7EEFF401B8442E5
:10550800FAD838BD000000207047436A10B59A6A7F
:1055180012F0500F1BD19A6A42F400729A621A680C
:10552800926802F46022B2F5602F0CD1DA6852B9A1
:105538009A6A22F480729A629A6AD2045EBF9A6A60
:1055480042F001029A621846FFF7DEFF10BD1B6A9F
:10555800BDE810401B6B1847704708B5406AFFF755
:10556800FBFF08BD7047406A08B5836A43F04003F3
:105578008362C36A43F00403C362FFF7F3FF08BD05
:10558800002373B5019390F82430012B74D00123C4
:105598004D6880F82430062D02684FEA85030C68B0
:1055A80025D82B441F25566B053B9D4026EA05054B
:1055B80004FA03F32B435363092C4FEA44038D6821
:1055C8002FD907262344D1681E3B9E4021EA0601B5
:1055D80005FA03F30B43D360A4F11003012B2BD975
:1055E8000023002280F82420184602B070BD0C2D3C
:1055F8000BD82B441F25166B233B9D4026EA050537
:1056080004FA03F32B431363D6E72B441F25D66A0A
:10561800413B9D4026EA050504FA03F32B43D36278
:10562800CAE70726116923449E4021EA060105FAC4
:1056380003F30B431361CFE7104B9A4216D19368DB
:105648001B02CDD49368102C43F400039360C7D198
:105658000B4B0C4A1B68B3FBF2F20A23534301932A
:10566800019B002BBCD0019B013BF8E7836A43F008
:10567800200383620123B4E70223B5E70024014035
:105688000002002040420F00002373B50193036815
:1056980004469A68D20702D5002002B070BD9A6805
:1056A80042F001029A60124B124A1B68B3FBF2F3F4
:1056B8000193019BC3B9FFF70FFF064623689D6856
:1056C80015F00105E8D1FFF707FF801B0228F5D97F
:1056D800A36A84F8245043F01003A362E36A01200C
:1056E80043F00103E362D8E7019B013BE0E700BF19
:1056F8000002002040420F002DE9D8419046404B5F
:10570800026804469A420F4602D03E498A4203D1B3
:105718005B6813F4702F6ED194F82430012B6CD091
:105728000123204684F82430FFF7AEFF0646002800
:105738005DD1A06A216820F47060324B20F001002E
:1057480040F480709942A06204D12D4A536813F442
:10575800702F3ED1A36A23F48013A3624B685A05C5
:1057680005D5A36A23F4405343F48053A362A36A84
:10577800206A13F4805318BFE36A3A4618BF23F02F
:105788000603E362002384F824301F4B4C31836204
:105798001E4BC3621E4B03636FF0020341F84C3C7F
:1057A80051F8443C43F4807341F8443C434600F0CC
:1057B800EDF923689A6802F46022B2F5602F9A68BE
:1057C8000CBF42F4A00242F480129A603046BDE851
:1057D800D881A36A43F48013A36253685B0541BF71
:1057E800A06A20F4405040F48050A062BFE7002334
:1057F80084F82430EAE70126E8E70226E6E700BF56
:105808000024014000280140135500086355000892
:105818006F55000838B5036804469A68D20701D462
:10582800002038BD9A6822F001029A60FFF754FE02
:10583800054623689B68DB07F2D5FFF74DFE401B42
:105848000228F6D9A36A012043F01003A362E36A91
:1058580043F00103E36238BDF8B50446002877D069
:10586800836A23B9C36280F8243003F019F820460C
:10587800FFF7D0FFA36A13F010036BD1002869D19A
:10588800A26A374922F4885222F0020242F0020248
:10589800A26294E824008A42E16904D1B1F5402F5C
:1058A80008BF4FF40021E66845EA46052943A56884
:1058B800B5F5807F35D0012D08BF4FF48073676937
:1058C800012F06D17EBBA669013E43EA463343F465
:1058D80000635668B5F5807F26F4694643EA0603F7
:1058E800536096681F4B03EA060343EA010393607B
:1058F80001D0012D20D12369013B1B05D56A25F470
:1059080070052B43D3629268174B1340994215D107
:105918000023E362A36A23F0030343F00103A362B5
:10592800F8BD2B46CBE7A66A46F02006A662E66AD3
:1059380046F00106E662CCE70023DFE7A36A23F01E
:10594800120343F01003A362E36A43F00103E36226
:105958000120F8BDA36A43F01003A362F8E700BF73
:10596800003C0140FDF7E1FFFE0E1FFF002373B569
:10597800019390F824300446012B5AD0012380F873
:105988002430FFF747FF0546002832D1A36A0220DA
:1059980023F4885323F0020343F00203A362264B47
:1059A8001E6800F0AFFFB6FBF0F040000190019BCD
:1059B8001BBB2046FFF768FE2268936843F0080384
:1059C8009360FFF789FD064623689A68120718D482
:1059D8009A6842F004029A60FFF77EFD0646236843
:1059E8009B685B071FD4A36A23F0030343F00103FA
:1059F800A362002384F8243012E0019B013B019349
:105A0800D5E7FFF769FD801B0A28DDD9A36A0125C0
:105A180023F0120343F01003A362002384F8243018
:105A2800284602B070BDFFF757FD801B0A28D6D95B
:105A3800ECE70225F4E700BF00020020074A000255
:105A4800D36800F4E06023F4E0631B041B0C43F00C
:105A5800BF6343F400330343D360704700ED00E0B5
:105A6800174B30B5DC68C4F30224C4F10703251DC5
:105A7800042B28BF0423062D4FF0010598BF0024EE
:105A880005FA03F303F1FF3388BF033C1940A14033
:105A980005FA04F4013C2240002842EA01024FEAD8
:105AA8000212AFBF00F16040064B00F00F00D2B207
:105AB800A5BFD2B200F561401A5480F8002330BD6A
:105AC80000ED00E014ED00E00123420900F01F00A2
:105AD80003FA00F0014B43F82200704700E100E0B0
:105AE8000138B0F1807F0AD2F021064B064A58608F
:105AF80082F823100020072298601A60704701205E
:105B0800704700BF10E000E000ED00E010B500288D
:105B180032D00168194B1424994225D8184AA3F2A7
:105B280007430A44B2FBF4F2920002648468C36338
:105B380043680A682343C46822F47F5223430469F4
:105B480022F0300223434469234384692343C46910
:105B5800234313430B600122002380F82120836331
:105B680080F82030184610BD064B0B44B3FBF4F305
:105B78009B000364044BD9E7012010BD07040240D1
:105B8800F8FFFDBFF8FBFDBF00040240F0B590F838
:105B98002040012C35D0012490F8215080F8204075
:105BA800A5424FF000064FF0020428D180F82140AA
:105BB800046886632668076C26F001062660C66BB3
:105BC800BD407560636043680568102BC36A0BBFEE
:105BD800A260A160E160E2604BB1236843F00E036C
:105BE80023602B68002043F001032B60F0BD23687D
:105BF80023F004032360236843F00A03F0E780F8E6
:105C080020600220F0BD000090F8213010B5022B72
:105C180003D004238363012010BD03681A6822F0AF
:105C28000E021A601A6822F001021A60294A934289
:105C380024D902F56272934219D01432934218D0D3
:105C48001432934217D0143293420CBF4FF480534E
:105C58004FF48033204A53600123002480F8213018
:105C6800436B80F820409BB39847204610BD012322
:105C7800F0E71023EEE74FF48073EBE717498B4208
:105C880016D014318B4215D014318B4214D01431F4
:105C98008B4214D014318B4214D014318B4214D05F
:105CA800934214BF4FF480334FF080730C4AD2E70D
:105CB8000123FBE71023F9E74FF48073F6E74FF46D
:105CC8008053F3E74FF48033F0E74FF48013EDE7A8
:105CD800184610BD8000024000040240080002403F
:105CE8000000024070B40425C66B026C3468036877
:105CF80095402542196855D04D0753D51A68960620
:105D08005EBF1A6822F004021A60604A93421FD9E3
:105D180002F56272934214D01432934213D01432B3
:105D2800934212D0143293420CBF4FF480434FF485
:105D38008023574A5360C36A002B00F0A58070BCCB
:105D480018470423F5E74023F3E74FF48063F0E7AF
:105D580050498B4216D014318B4215D014318B42E6
:105D680014D014318B4214D014318B4214D0143116
:105D78008B4214D0934214BF4FF480234FF08063BA
:105D8800454AD7E70423FBE74023F9E74FF480634C
:105D9800F6E74FF48043F3E74FF48023F0E74FF43E
:105DA8008003EDE702259540254257D08D0755D54C
:105DB8001A68940606D41A6822F00A021A600122A8
:105DC80080F82120314A93421ED902F5627293422B
:105DD80013D01432934212D01432934211D0143299
:105DE80093420CBF4FF400534FF40033284A5360DA
:105DF800002380F82030836A9EE70223F6E72023F9
:105E0800F4E74FF40073F1E722498B4216D01431BE
:105E18008B4215D014318B4214D014318B4214D0DC
:105E280014318B4214D014318B4214D0934214BFD6
:105E38004FF400334FF00073174AD8E70223FBE70B
:105E48002023F9E74FF40073F6E74FF40053F3E724
:105E58004FF40033F0E74FF40013EDE708259540C1
:105E6800254211D009070FD5196821F00E011960D4
:105E7800012303FA02F27260836380F82130002361
:105E880080F82030036B57E770BC704780000240F1
:105E9800000402400800024000000240114AD36892
:105EA80013F0100305D01049CB6943F00203CB610E
:105EB8001023D268500706D50B4943F00403CA697A
:105EC80042F00102CA61074AD169C90708D50648E4
:105ED800C16941F00401C161D16921F00101D161B9
:105EE800D36070470020024060040020064B186908
:105EF80010F0800007D0054A5A6002F188325A60D3
:105F08001869C0F3C010704700200240230167459C
:105F1800034A0020136943F080031361704700BFF0
:105F280000200240F8B50646FFF7D6FA114C07469E
:105F38002546E368D80712D4E368990644BF2023AE
:105F4800E360EB68DA0606D4EB69DB0703D4E8689C
:105F580010F0040002D0FFF7A1FF0120F8BD731C68
:105F6800E7D00EB90320F8BDFFF7B6FAC01B86428A
:105F7800DFD2F7E7002002402DE9F84F1F4C994681
:105F8800237E0546012B0F46904633D001234CF261
:105F980050302376FFF7C6FF40BB012D03D0022DFA
:105FA8000CBF022504250026B246DFF854B03201A2
:105FB80040464946FEF73CF9C4F81CA0DBF810300F
:105FC80080B243F00103CBF8103027F816004CF2EA
:105FD8005030FFF7A7FFDBF8103023F00103CBF8B0
:105FE800103018B90136F3B29D42E0D80023237669
:105FF800BDE8F88F0220BDE8F88F00BF60040020DC
:10600800002002400022064BDA61064B1A6942F072
:1060180004021A611A6942F040021A61704700BF0F
:1060280060040020002002400022064BDA61064B83
:106038001A6942F002021A6158611A6942F0400274
:106048001A61704760040020002002402DE9F041E9
:10605800234D07462B7E8846012B3DD0012403683B
:106068002C76022B4CF2503013D1FFF75BFF20B196
:10607800012000232B76BDE8F081FFF7C3FF4CF227
:106088005030FFF74FFF174A136923F004031361D9
:10609800EFE7FFF747FF0028EAD14FF0FF33C8F8D2
:1060A80000302046BE680F4CFA68BB6803EBC22379
:1060B8009E42DED23046FFF7B7FF4CF25030FFF772
:1060C80031FF236923F00203236110B1C8F800608F
:1060D800CFE706F50066E7E70220BDE8F08100BFDC
:1060E80060040020002002402DE9F74F00221646E8
:1060F8006C4F6D4BDFF8B8E1DFF8B8C14FF001081D
:106108000C6808FA06F808EA0404A04540F08580FF
:106118004D68122D00F0B78000F28D80022D00F03E
:10612800AF8000F28180002D00F09180012D00F0F9
:10613800A5804FF00F09FF2C93BF824606F18045DA
:10614800083DD0F800B092BFB500D0F804B0AD005B
:1061580009FA05F82BEA080802FA05F588BF00F1E4
:10616800040A48EA0505CAF80050D1F804A01AF054
:10617800805F52D0BD6926F0030845F00105BD6176
:10618800BD6908F1804805F00105019508F58038DA
:1061980006F0030B019D4FEA8B0BD8F8085009FA5B
:1061A8000BF925EA0909414DA84271D005F580652A
:1061B800A8426FD005F58065A8426DD005F58065C9
:1061C800A8426BD005F58065A84269D070450CBF20
:1061D8000525062505FA0BF545EA0905C8F808500E
:1061E8001D681AF4803F14BF2543A5431D605D68F0
:1061F8001AF4003F14BF2543A5435D609D681AF457
:10620800801F14BF2543A5439D60DD681AF4001F55
:1062180014BF2C4325EA0404DC600136102E7FF4F9
:106228006DAF03B0BDE8F08F032D25D0112D80D1BF
:10623800CA6804327DE7654509D012D8DFF878903E
:106248004D4504D009F580394D457FF472AF8A6811
:10625800E2B1012A0CBFC0F81080C0F814800822EF
:1062680067E7DFF858904D45F1D009F580394D457D
:10627800EDD0A9F58019E7E700225AE7CA6858E780
:10628800CA68083255E7CA680C3252E7042250E758
:1062980000259FE701259DE702259BE7032599E750
:1062A800042597E70010024000040140000801405F
:1062B800001C0140000021100000111000003110E6
:1062C8008368194214BF0120002070470AB1016198
:1062D80070470904FBE7C3685940C1607047000074
:1062E80003682DE9F341DB07054610D42B689F07A7
:1062F8005ED42B68190700F195802B685A0700F1C6
:10630800BF80EA69002A40F02D81002014E0904CFB
:10631800636803F00C03042B07D0636803F00C03D5
:10632800082B0CD16368DE0309D523689C03DDD5EF
:106338006B68002BDAD1012002B0BDE8F0816B68F0
:10634800B3F5803F10D1236843F480332360FFF70F
:10635800C3F8064623689803C8D4FFF7BDF8801B26
:106368006428F7D90320E7E79BB9236823F480332F
:106378002360236823F480232360FFF7ADF80646E3
:1063880023689903B2D5FFF7A7F8801B6428F7D9CB
:10639800E8E7B3F5A02F236803D143F480232360F3
:1063A800D1E723F480332360236823F48023CDE7E7
:1063B800674C636813F00C0F07D0636803F00C0395
:1063C800082B10D16368DA030DD423689B0702D524
:1063D8002B69012BAFD123686A6923F0F80343EADC
:1063E800C203236085E72A695A4B6AB101221A6001
:1063F800FFF772F8064623689F07ECD4FFF76CF89E
:10640800801B0228F7D9ADE71A60FFF765F8064642
:10641800236898077FF56DAFFFF75EF8801B0228A9
:10642800F6D99FE7AA694A4C4B4BDAB101221A60A8
:10643800FFF752F80646636A9B070DD54FF4FA52E8
:10644800464B1B68B3FBF2F3019300BF019B5A1E36
:106458000192002BF9D150E7FFF73EF8801B022884
:10646800E9D97FE71A60FFF737F80646636A9F079E
:106478007FF543AFFFF730F8801B0228F6D971E7A4
:10648800334CE369D80024D40127E36943F08053EF
:10649800E361E36903F080530093009B304E336857
:1064A800D90518D5EB68012B26D1236A43F00103DF
:1064B8002362FFF711F841F288368046236A9B076A
:1064C8003FD5002F3FF41DAFE36923F08053E3610C
:1064D80017E70027E2E7336843F480733360FEF779
:1064E800FBFF80463368DA05DCD4FEF7F5FFA0EB46
:1064F80008006428F6D935E7ABB9236A41F2883831
:1065080023F001032362236A23F004032362FEF7C6
:10651800E3FF0646236A9807D3D5FEF7DDFF801B05
:106528004045F7D91EE7052B236A03D143F004033E
:106538002362BAE723F001032362236A23F00403EA
:10654800B6E7FEF7C9FFA0EB0800B042B6D909E7E5
:106558000010024000004242800442420002002033
:1065680000700040224C636803F00C03082B3FF4D2
:10657800E2AE00231F4E022A33602BD1FEF7ACFF98
:106588000746236899011FD42B6AB3F5803F05D1CC
:106598006268A96822F400320A436260696A626824
:1065A8000B4322F474121343636001233360FEF734
:1065B80093FF054623689A013FF5A7AEFEF78CFFC7
:1065C800401B0228F6D9CDE6FEF786FFC01B02283D
:1065D800D7D9C7E6FEF780FF054623689B017FF5FC
:1065E80094AEFEF779FF401B0228F6D9BAE600BF41
:1065F800001002406000424230B5194B87B002AC2F
:1066080003F11005224618685968083303C2AB42E3
:106618001446F7D101238DF80430022311498DF86F
:1066280005304B6803F00C02082A17D1C3F38342E4
:1066380006A80244DB0312F8102C0CD54B680A4854
:10664800C3F34043504306AA134413F8143CB0FB69
:10665800F3F007B030BD05485043FAE70248F8E7C1
:1066680040BF00080010024000127A0000093D00F7
:10667800544A2DE9F0411368054603F007038B429D
:106688000E462AD329688C0734D4CA0747D44D4A02
:10669800136803F007039E42C0F082802A684A4CC0
:1066A80012F0040F40F08780130706D563682A6943
:1066B80023F4605343EAC2036360FFF79DFF6368F6
:1066C800424AC3F30313D35CD840414B18600020FF
:1066D800FEF7C0FE0020BDE8F081136823F0070331
:1066E8000B431360136803F007039942CAD00120D3
:1066F800BDE8F081344B11F0040F1EBF5A6842F414
:10670800E0625A60080742BF5A6842F460525A6011
:106718005A68A86822F0F00202435A60B5E76A682E
:10672800294C012A23681CD113F4003FDFD0636889
:1067380041F2883823F0030313436360FEF7CCFE6D
:106748006B680746012B14D1636803F00C03042B14
:106758009DD0FEF7C1FEC01B4045F5D90320BDE81A
:10676800F081022A02D113F0007FDFE713F0020F55
:10677800DCE7022B0FD1636803F00C03082B86D0EB
:10678800FEF7AAFEC01B4045F5D9E7E7FEF7A4FED1
:10679800C01B4045E2D8636813F00C0FF6D176E7CA
:1067A800136823F0070333431360136803F00703E8
:1067B8009E429CD172E76368E96823F4E0630B4367
:1067C800636071E70020024000100240AFBF00087C
:1067D80000020020044B054A5B68C3F30223D35C24
:1067E800034A1068D840704700100240BFBF000835
:1067F80000020020044B054A5B68C3F3C223D35C44
:10680800034A1068D840704700100240BFBF000814
:106818000002002003682DE9F341D907054620D579
:10682800354CE369DA0032D40127E36943F0805339
:10683800E361E36903F080530193019B2F4E3368B2
:10684800DB0526D5236A13F4407336D1236A6A68B8
:1068580023F44073134323621FB1E36923F0805389
:10686800E3612868830706D5234AA968536823F497
:1068780040430B43536010F010001BD01E4A696957
:106888005368002023F480030B43536012E0002771
:10689800D4E7336843F480733360FEF71DFE804607
:1068A8003368D805CED4FEF717FEA0EB080064289D
:1068B800F6D9032002B0BDE8F0816A6802F440729C
:1068C8009342C3D001200E4A236A1060002023F4AB
:1068D800407110602162D907B8D5FEF7FDFD41F27D
:1068E80088380646236A9A07B0D4FEF7F5FD801B60
:1068F8004045F7D9DDE700BF0010024000700040B6
:1069080040044242024670B53B4B86B002AD03F1EB
:1069180010062C4618685968083303C4B342254644
:10692800F7D101238DF804300223501E8DF805306D
:106938000F285ED8DFE800F032515D2D5D5D5D2DDA
:106948005D5D5D5D5D5D5D082C4B5968186810F0F4
:10695800807037D0C1F3834206A8024412F8100CA5
:10696800CA0341BF5A6806A9C2F34042521844BF3D
:1069780012F8141C224A5B684CBFB2FBF1F2214AA0
:106988005B0202FB00F01DD403234000B0FBF3F0D0
:1069980018E006B0BDE87040FFF72EBE40F20231A5
:1069A800164A136A1940B1F5817F1FD003F440736A
:1069B800B3F5007F08D149F64040536A13F0020F3F
:1069C80008BF002006B070BDB3F5407F11D1136831
:1069D8004FF2244013F4003FF2E7FFF70BFF074B99
:1069E8005B68C3F3813301335B00CFE74FF40040AA
:1069F800E8E70020E6E700BF50BF000800100240AB
:106A080000127A0000093D007047704770477047D0
:106A1800036810B51A69044691070ED5DA6892071B
:106A28000BD56FF002021A6101229B6902779B075E
:106A380077D0FFF7EAFF0023237723681A69500706
:106A480010D5DA6851070DD56FF004021A610222D9
:106A58009B69227713F4407F204668D0FFF7D5FF63
:106A68000023237723681A6912070FD5DA681007FD
:106A78000CD56FF008021A610422DB6922779907A6
:106A880020465AD0FFF7C1FF0023237723681A69ED
:106A9800D20610D5DA68D0060DD56FF010021A614B
:106AA8000822DB69227713F4407F20464BD0FFF79A
:106AB800ACFF0023237723681A69D10708D5DA6861
:106AC800D20705D56FF0010220461A6101F038F9A6
:106AD80023681A69100608D5DA68110605D56FF01B
:106AE800800220461A6100F0BEF823681A6952062F
:106AF80008D5DA68500605D56FF0400220461A61BD
:106B0800FFF785FF23681A69910622D5DA6892068D
:106B18001FD56FF020022046BDE810401A6100F032
:106B2800A1B8FFF771FF2046FFF770FF83E7FFF773
:106B38006BFF2046FFF76AFF92E7FFF765FF2046E5
:106B4800FFF764FFA0E7FFF75FFF2046FFF75EFF50
:106B5800AFE710BD244A0368904212D002F50062E4
:106B680090420ED0B0F1804F0BD0A2F598329042EF
:106B780007D002F58062904203D002F5806290420D
:106B88001DD14A6823F070031343174A904212D06C
:106B980002F5006290420ED0B0F1804F0BD0A2F502
:106BA8009832904207D002F58062904203D002F5F5
:106BB8008062904203D1CA6823F4407313434A6940
:106BC80023F08003134303608B68C3620B688362FE
:106BD800054B984203D003F50063984201D10B6935
:106BE8000363012343617047002C014010B504463C
:106BF800A0B190F83D3003F0FF021BB980F83C20AB
:106C080001F0BEFE0223206884F83D30211DFFF705
:106C1800A1FF0123002084F83D3010BD012010BDE4
:106C280090F83C3010B5012B4FF0020318D080F8D3
:106C38003D3003680C685A68496822F070025A604F
:106C48005A6822435A609A6822F080029A609A68C9
:106C58000A439A60012380F83D30002380F83C30D5
:106C6800184610BD704770470368DA6822F49072BE
:106C7800DA605A6922F001025A61202380F83A301A
:106C8800704700002DE9F0470568C2682B69016963
:106C980023F4405313432B618368EA680B4341692B
:106CA80022F4B05222F00C020B431343EB606B69E1
:106CB800826923F4407313436B61404B81469D42C4
:106CC8004FF0190446D1FFF795FD04FB00F3D9F8FE
:106CD80004604FF06408B600B3FBF6F3B3FBF8F3B7
:106CE8001E01FFF787FD6043D9F804309B00B0FB15
:106CF800F3F7FFF77FFD6043D9F804309B00B0FB42
:106D0800F3F3B3FBF8F308FB13731B013233B3FB44
:106D1800F8F303F0F007FFF76DFD6043D9F804209E
:106D28009200B0FBF2FAFFF765FD6043D9F8043032
:106D38009B00B0FBF3F3B3FBF8F308FB13A31B01B1
:106D48003233B3FBF8F303F00F033B433344AB6038
:106D5800BDE8F087FFF73EFD04FB00F3D9F80460B7
:106D68004FF06408B600B3FBF6F3B3FBF8F31E016B
:106D7800FFF730FD6043D9F804309B00B0FBF3F710
:106D8800FFF728FD6043D9F804309B00B0FBF3F30C
:106D9800B3FBF8F308FB13731B013233B3FBF8F3AF
:106DA80003F0F007FFF716FD6043D9F804209200BE
:106DB800B0FBF2FAFFF70EFDB7E700BF003801405D
:106DC800F8B504460E4617461D4621680B6836EA94
:106DD800030301D10020F8BD6B1CF7D095B92368D7
:106DE8000320DA6822F4D072DA605A6922F00102CC
:106DF8005A61202384F8393084F83A30002384F823
:106E08003830F8BDFEF768FBC01B8542DDD2E6E7E7
:106E180010B5044640B390F8393003F0FF021BB9AF
:106E280080F8382001F0C0FD2423226884F8393026
:106E3800D368204623F40053D360FFF723FF236869
:106E480000201A6922F490421A615A6922F02A0233
:106E58005A61DA6842F40052DA602023E06384F869
:106E6800393084F83A3010BD012010BD2DE9F041C9
:106E78001F4690F839300446202B0D4690464ED1D7
:106E8800002949D0002A47D090F83830012B46D045
:106E9800012380F838300023C363212380F8393078
:106EA800FEF71AFB0646A4F82480A4F82680E38C93
:106EB8009BB26BB93B46324640212046FFF780FF24
:106EC800A8B9202384F8380084F83930BDE8F08167
:106ED800E38C3246013B9BB2E384A3688021B3F57F
:106EE800805F20463B460ED1FFF76AFF10B10320B2
:106EF800BDE8F0812B882268C3F308035360236937
:106F080043B90235D3E7FFF75BFF0028EFD12368C9
:106F18002A785A600135CAE70120BDE8F0810220CD
:106F2800BDE8F08138B50446134694F83920202A84
:106F38002AD139B333B394F83820012A24D0012256
:106F4800002584F838202122E384206BE56384F847
:106F580039200E4AA384216282620D4A4563C262C7
:106F68000C4A026322680432FEF710FE6FF04002FA
:106F7800236828461A605A6984F8385042F080021B
:106F88005A6138BD012038BD022038BD3370000871
:106F9800617000082D710008134690F83A2073B507
:106FA800202A054638D1002934D0002B32D090F859
:106FB8003820012A30D00122002480F838202222EB
:106FC80081628385C46380F83A20406B134A2E6837
:106FD8008262134A4463C262124A02630A46311D3E
:106FE800FEF7D4FD20462B6801941A6801925A686E
:106FF80085F838400192019ADA6842F48072DA60C2
:107008005A6942F001025A615A6942F040025A61D3
:1070180002B070BD0120FBE70220F9E76B700008A1
:10702800217100082D710008704708B50368426A8D
:107038001B6813F020030AD1D38413685A6922F01D
:1070480080025A61DA6842F04002DA6008BD1046F0
:10705800FFF7EAFF08BD704708B5406AFFF7FBFF76
:1070680008BD08B50368426A1B6813F0200310D1F5
:10707800D3851368D96821F48071D960596921F0E2
:1070880001015961596921F040015961202382F8B1
:107098003A30104601F0A6FD08BD90F83A3010B518
:1070A800222B36D183680169B3F5805F0268836A51
:1070B80023D15268E9B9C2F3080223F8022B83628C
:1070C800C48D013CA4B2C4858CB90368DA6822F087
:1070D8002002DA60DA6822F48072DA605A6922F0F3
:1070E80001025A61202380F83A3001F07BFD00202C
:1070F80010BDD2B223F8012BE1E721B9591C52681F
:1071080081621A70DCE75268591C816202F07F02C2
:10711800F7E7022010BD704708B5406AFFF7FBFF8C
:1071280008BD7047416A08B50B685A6991F839007B
:1071380021280AD1120608D50022CA84DA6822F06A
:10714800C002DA60202281F839205B6991F83A2080
:10715800222A06D15B0604D500230846CB85FFF713
:1071680083FDCB6B084643F01003CB63FFF7D9FFD1
:1071780008BD0000036870B51A6804461607D96888
:107188005D6907D196065AD58D0658D5BDE8704079
:10719800FFF783BF15F0010502D111F4907F4ED09F
:1071A800D30705D5CE0542BFE36B43F00103E36384
:1071B800500704D51DB1E36B43F00203E363930763
:1071C80004D51DB1E36B43F00403E363160704D54C
:1071D8001DB1E36B43F00803E363E36B002B66D058
:1071E800950604D5880602D52046FFF756FF236882
:1071F80020465D69E26B110702D415F040051AD0EC
:10720800FFF732FD23685A69520610D55A69606B38
:1072180022F040025A6150B1254B4363FEF7F4FC5B
:10722800002844D0606BBDE87040436B1847204687
:10723800FFF777FF70BDFFF774FFE56370BD1606B3
:1072480027D50D0625D594F83920212A2FD1A268F3
:10725800B2F5805F226A17D11188C1F3080159601D
:10726800216979B902322262E28C013A92B2E2844F
:10727800EAB9DA6822F08002DA60DA6842F040029D
:10728800DA6070BD0132EEE7511C216212785A6053
:10729800EAE750060BD54A0609D5DA68204622F0F7
:1072A8004002DA60202384F83930FFF7BDFE70BD54
:1072B800BD72000808B50023406AC385C384FFF780
:1072C80030FF08BD70B50022054604212448FEF7AA
:1072D800FDFF1024224E012208213046FEF7F6FF5A
:1072E8002B044CBF0122002210213046FEF7EEFF8E
:1072F800013C002208213046FEF7E8FF6D0014F03B
:10730800FF04ADB2E7D101224FF400411548FEF762
:10731800DDFF0A2000F038FD22464FF400411148F5
:10732800FEF7D4FF012204210D48FEF7CFFF2246C5
:1073380010210B48FEF7CAFF01224FF4004109480B
:10734800FEF7C4FF224604210548FEF7BFFF224688
:10735800BDE870404FF400410248FEF7B7BF00BFD8
:10736800002001400014014084B02DE9F84F0AAC18
:1073780084E80F000E9EBDF83C7000223946814615
:1073880030469DF84050BDF82CA0DDF83080BDF89F
:1073980034B0FEF79BFF0120FEF7A4F80824AD00E7
:1073A800EDB215F0010218BF012259464046FEF71A
:1073B8008DFF012251464846FEF788FF0120FEF75F
:1073C80091F8002251464846FEF780FF013C012013
:1073D800FEF788F814F0FF044FEA5505E1D122467C
:1073E80051464846FEF772FF22464FF40041404698
:1073F800FEF76CFF0520FEF775F839460122304686
:10740800FEF764FF0120FEF76DF822463946304644
:10741800BDE8F84F04B0FEF759BF10B5FF23044686
:10742800221AD2B2914201D8184610BD14F8012B85
:107438005340082213F0800F02F1FF324FEA430352
:1074480018BF83F0310312F0FF02DBB2F2D1E7E795
:1074580030B5FF2305462C1AE4B2A14203D89B1A83
:107468005842584130BD15F8014B6340082413F0C9
:10747800800F04F1FF344FEA430318BF83F0310350
:1074880014F0FF04DBB2F2D1E5E784B08DE80F0019
:107498009DF818209DF81C3002981A4112F001023C
:1074A800BDF80C1018BF012204B0FEF70FBF000092
:1074B80084B02DE9F04F85B00EAC84E80F00129D22
:1074C800BDF84C600022314680462846BDF83C9005
:1074D800FEF7FCFE0A2000F057FC00270DF1480BD0
:1074E8000DF1640A9DF85030FCB202931295ADF884
:1074F8004C6003949BE803008DE80300CDF83880C6
:10750800ADF83C900EAB0FCBFFF7BFFF9DF86C308A
:10751800039402939AE803008DE8030015AB0FCBA0
:10752800FFF7B3FF9DF888300394029320AB93E8EC
:1075380003008DE803001CAB0FCBFFF7A6FF9DF8F7
:10754800A4300394029327AB93E803008DE803006B
:1075580023AB0FCBFFF799FF9DF8C030039402933C
:107568002EAB93E803008DE803002AAB0FCBFFF79F
:107578008CFF012249464046FEF7A8FE0A2000F08B
:1075880003FC0137002249464046FEF79FFE082FBC
:10759800A8D100224FF400410948FEF797FE314672
:1075A80001222846FEF792FE0A2000F0EDFB002299
:1075B8003146284605B0BDE8F04F04B0FEF786BE58
:1075C800000C0140F0B5214C214E25460FCE0FC5C9
:1075D80096E803001F4F04F11C0685E803000FCF4F
:1075E8000FC697E803001C4F86E803000FCF04F18D
:1075F80038060FC697E80300184F86E803000FCF38
:1076080004F154060FC697E80300154F86E80300F7
:107618000FCF04F170060FC697E803000023A1B04E
:1076280086E803007C2229466846237684F83430AD
:1076380084F8503084F86C3084F8883001F0FEFF0C
:1076480094E80F00FFF734FF21B0F0BDE0040020FC
:10765800700100208801002028010020400100203E
:107668005801002070B50223044601250020E607D2
:1076780048BF05FA03F603F1010348BF80190E2B32
:107688004FEA5404F3D10124CD0748BF04FA03F5A7
:1076980003F1010348BF4019162B4FEA5101F3D1FA
:1076A800D30748BF00F5800070BDF0B5064601203D
:1076B800022407469DF8145016F0010F18BF07FA68
:1076C80004FE04F1010418BF70440E2C4FEA56065C
:1076D800F2D10126CF0748BF06FA04F704F10104E6
:1076E80048BFC019122C4FEA5101F3D1D70744BF44
:1076F80000F580201324DE0742BF012303FA04F4B7
:107708000019EC0748BF00F500209DF81830A907BC
:1077180048BF00F580106A0748BF00F50010DB0776
:1077280048BF00F58000F0BD2DE9F74F16464FF42D
:107738007A729DF838B0002502FB0BF28246DDE92B
:107748000C011F46D317FDF7FDFC0F9A2B46804608
:107758008946FDF7F7FCC0EB40144FF47A7200231A
:1077680000EB840439463046FDF7ECFCFCF7EEFEEE
:107778004FF47A7206460F46002340464946FDF705
:10778800E1FCFCF7E3FE02460B4630463946FDF7BE
:107798003DF800221A4BFDF739F80F460646FDF76B
:1077A800E3F91FFA80F84046FCF790FE0B460246C4
:1077B80039463046FCF74CFDFDF7F6F9E400A4B273
:1077C80006462046FDF7FAFA01463046FDF74AFB21
:1077D800FDF798FC2A46414680B2FFF743FF022393
:1077E8000646009301952B46012259462046FFF78D
:1077F8005CFF8AE84100504603B0BDE8F08F00BF47
:1078080000408F4084B02DE9F04F85B00EAC84E87D
:107818000F00179BBDF83C80C3F30A0ABDF8583027
:10782800109C0193159BBDF8445023F07F430293AD
:10783800149B129E23F07F43BDF84C7000224146F2
:1078480003938146FEF742FD002229462046FEF7B3
:107858003DFD002239463046FEF738FD4FF00B0B50
:107868001AF4806218BF012229462046FEF72EFD31
:10787800322000F089FA012241464846FEF726FDEB
:10788800322000F081FA002241464846FEF71EFDEC
:10789800BBF1010B4FEA4A0AE2D1012239463046D0
:1078A800FEF714FD322000F06FFA5A46394630468A
:1078B800FEF70CFD4FF0100A019B294613F4004215
:1078C80018BF01222046FEF701FD322000F05CFAC5
:1078D800012241464846FEF7F9FC322000F054FAEE
:1078E800002241464846FEF7F1FC019BBAF1010A25
:1078F8004FEA43039BB20193DED101223946304659
:10790800FEF7E4FC322000F03FFA52463946304692
:10791800FEF7DCFC4FF0180A029B294613F400021C
:1079280018BF01222046FEF7D1FC322000F02CFAC5
:10793800012241464846FEF7C9FC322000F024FAED
:10794800002241464846FEF7C1FC029BBAF1010AF3
:107958004FEA430323F07F430293DDD101223946E6
:107968003046FEF7B3FC322000F00EFA5246394694
:107978003046FEF7ABFC4FF0180A039B294613F478
:10798800000218BF01222046FEF7A0FC322000F0BA
:10799800FBF9012241464846FEF798FC322000F0E8
:1079A800F3F9002241464846FEF790FC039BBAF1E2
:1079B800010A4FEA430323F07F430393DDD1524684
:1079C80029462046FEF782FC394601223046FEF75A
:1079D8007DFC322000F0D8F952463946304605B0D1
:1079E800BDE8F04F04B0FEF771BC000000000000D5
:1079F8002DE9F043304C95B0264608AD0FCE0FC5A3
:107A080096E80300183485E803000FCC0EAD0FC5C7
:107A180094E8030024A3D3E9002341F288394FF006
:107A28000208002785E8030041F2C2340325234EEB
:107A380006A8CDF80C90CDF80880CDE90067FFF7CF
:107A480073FE069B05950393079B049402930CAB66
:107A580093E803008DE8030008AB0FCBFFF7D2FED5
:107A68000120FDF73FFD12A3D3E9002306A8CDF8B6
:107A78000C90CDF80880CDE90067FFF755FE069B0E
:107A880005950393079B0494029314AB13E9030031
:107A98008DE803000EAB0FCBFFF7B4FE012015B045
:107AA800BDE8F043FDF71EBD60558FCE0000000015
:107AB800A0B483EA0000000060BF0008005A620218
:107AC80038B500231A4CBE2223601A4B0546A36022
:107AD8000123E36043705D2383705E230270C370EB
:107AE800FEF704FA14492046FEF7B0FA18B1134815
:107AF80002F08CFAFEE704462B195B782A5D04F144
:107B0800006102EB032292B2002301F5FF2101205C
:107B1800FEF732FA20B1A421094802F003FAFEE781
:107B28000234602CE8D1BDE83840FEF7F1B900BF57
:107B38002404002000F807083404002090BF00083F
:107B48009EBF000808B5FFF7BBFF08BD002303F17F
:107B5800006202F5FF221188C1541288C11802334D
:107B6800C2F30722602B4A70F1D1704770B5244DDB
:107B78004FF480412846FEF7A3FB224C4FF4004106
:107B880084F840002846FEF79BFB1F4E84F841000E
:107B980001213046FEF794FB022184F8420030466A
:107BA800FEF78EFB802184F843001848FEF788FB17
:107BB80006F5006684F847004FF400713046FEF77A
:107BC8007FFB4FF4806184F846003046FEF778FB6F
:107BD8004FF4006184F844003046FEF771FB4FF41F
:107BE800805184F845002846FEF76AFB4FF480610F
:107BF80084F848002846FEF763FB84F8490070BD06
:107C0800001001406C0500200018014000140140DC
:107C1800403810B50C460D2877D8DFE800F0071279
:107C28001920353C2D26434A5151515139B1012271
:107C38004FF480413548BDE81040FEF747BB0A467F
:107C4800F6E719B101224FF40041F3E70A46FAE7D3
:107C580019B1012201212E48EDE70A46FAE711B1D0
:107C680001220221F7E70A46FBE719B10122802128
:107C78002848E0E70A46FAE721B101224FF40071EB
:107C88002548D8E70A46F9E719B101224FF480617F
:107C9800F6E70A46FAE719B101224FF40061EFE767
:107CA8000A46FAE719B101224FF48051C2E70A46A1
:107CB800FAE719B101224FF48061BBE70A46FAE7F7
:107CC80091B1002220211448FEF700FB0022402138
:107CD8001148FEF7FBFA012280210F48FEF7F6FA59
:107CE80001224FF48071CBE7012220210A48FEF7D8
:107CF800EDFA012240210848FEF7E8FA22468021E1
:107D08000548FEF7E3FA2246EBE710BD00100140F4
:107D180000180140001401400020014010B5074C34
:107D2800A178601CFFF779FB84F85E00204601F01B
:107D3800E7FBBDE8104000F08BBF00BF80040020C7
:107D48000268084B9A420BD1074A13680133136043
:107D5800064A136801331360054A13680133136038
:107D6800704700BF00100040400400203C04002081
:107D78003804002010B514460A230248FFF776F8A5
:107D8800204610BDBC060020084A0949126882B086
:107D9800B2FBF1F20190019B53430193019B5A1EE0
:107DA8000192002BFAD102B0704700BF00020020F8
:107DB80040420F0010B596B0282200210CA801F00F
:107DC80048FC1422002101A801F043FC18220021DC
:107DD8000DEB020001F03DFC012310931023022457
:107DE80011934FF440130CA815930C941394FEF7B9
:107DF80077FA0F234FF4806201930023214601A8EC
:107E08000393049205930294FEF732FC4FF48043E7
:107E180006A806940893FEF7FDFC16B010BD0000F6
:107E28002DE9F04FB44D95B0FDF738FBFFF7C2FFD1
:107E38001022002110A801F00CFCAB69002243F0CD
:107E48004003AB61AB697F2103F040030993099BB1
:107E5800AB69AA4843F01003AB61AB69002403F097
:107E680010030A930A9BAB69012643F08003AB61B8
:107E7800AB69022703F080030B930B9BAB694FF0B0
:107E88000C0B43F00403AB61AB694FF00E0903F030
:107E980004030C930C9BAB694FF0070843F00803ED
:107EA800AB61AB694FF0030A03F008030D930D9B18
:107EB800AB6943F02003AB61AB6903F020030E9379
:107EC8000E9BAB6943F48073AB61AB6903F48073B9
:107ED8000F930F9BFEF7FAF900224FF6C04188482E
:107EE800FEF7F4F9002240F2F3318648FEF7EEF986
:107EF800002248F6FF718448FEF7E8F9002247F6A9
:107F0800FC718248FEF7E2F900224FF400418048F4
:107F1800FEF7DCF9002218217E48FEF7D7F97F2307
:107F280010A976481093119612941397FEF7DCF86F
:107F38004FF6C04310A972481093119612941397E4
:107F4800FEF7D2F840F2F33310A96E481093119659
:107F580012941397FEF7C8F810A96A48CDF840B0F4
:107F680011941294FEF7C0F848F6FF7310A96648FA
:107F78001093119612941397FEF7B6F84FF44053E6
:107F880010A96148109311941294FEF7ADF847F6C2
:107F9800FC7310A95D481093119612941397FEF77D
:107FA800A3F84FF4407310A95548109311941294F4
:107FB800FEF79AF84FF4004310A955481093079319
:107FC800119612941397FEF78FF8182210A95148AA
:107FD8001092119612941397FEF786F8602210A952
:107FE8004C48109211941294FEF77EF86A694FF487
:107FF800807332436A616A69474D32400892089A31
:10800800464A28462A604FF46022AB60EA61109421
:1080180011941294EE606C616C60C5F81090FDF7D5
:108028001BFC10A92846CDF8488010941196FDF73E
:10803800A7FA10A9284610961197FDF7A1FA10A9DA
:108048002846CDF844A01097FDF79AFACDF840A03D
:108058004FF0040A10A92846CDF844A0FDF790FA7D
:10806800CDF840A04FF0050A10A92846CDF844A045
:10807800FDF786FACDF840A04FF0060A10A9284669
:10808800CDF844A0FDF77CFA10A92846CDF840A009
:10809800CDF84480FDF774FACDF840804FF0080819
:1080A80010A92846CDF84480FDF76AFACDF840803B
:1080B8004FF0090810A92846CDF84480FDF760FA6A
:1080C8000A224FF00B0ACDF840804FF00D0810A996
:1080D800284611920692FDF753FA069A10A92846E7
:1080E8001092CDF844A0FDF74BFA10A92846CDF818
:1080F80044B0CDF840A013E0001002400018014041
:1081080000100140001C0140001401400020014003
:1081180000080140000C01404806002000240140EE
:10812800FDF72EFA10A92846CDF840B0CDF84480C6
:10813800FDF726FA10A92846CDF84080CDF84490DE
:10814800FDF71EFA4FF4E133DFF8A083D249404629
:1081580088E80A00C8F814B0C8F80840C8F80C4005
:10816800C8F81040C8F81840C8F81C40FEF750FE80
:1081780041F2DF52DFF878B3C84958468BE8060069
:10818800069A1094CBF80C201194CBF80840CBF841
:108198001840FEF72BFD10A9584610941194FEF7CD
:1081A8003FFD224621462520FDF75AFC2520FDF7F4
:1081B8008BFC224621463620FDF752FC3620FDF77F
:1081C80083FC224621465046FDF74AFC5046FDF7FF
:1081D8007BFC224621464846FDF742FC4846FDF70F
:1081E80073FC224621460F20FDF73AFC0F20FDF7CD
:1081F8006BFCAB4A21461268906801F00FFF3246CB
:10820800A8494046FEF7C8FEFFF7DCF922464FF4BE
:108218008041A548FEF75AF8079B22461946A2480E
:10822800FEF754F822463146A048FEF74FF822469A
:1082380039469E48FEF74AF822464FF480619C482A
:10824800FEF744F822464FF400619948FEF73EF8DD
:1082580022464FF400719648FEF738F822468021EE
:108268009448FEF733F832464FF480518E48FEF7B3
:108278002DF832464FF480618B48FEF727F82246E6
:1082880020218B48FEF722F8224640218848FEF735
:108298001DF8324680218648FEF718F832464FF41A
:1082A80080718348FEF712F83046FDF71BF9FFF797
:1082B8005DFCFFF79DFB48F20C00FFF703F84FF455
:1082C8002040FEF7FFFF40F6FF70FEF7FBFF41F28C
:1082D800FF30FEF7F7FF42F2FF40FEF7F3FF43F2ED
:1082E800FF50FEF7EFFF44F2FF60FEF7EBFF45F2A9
:1082F800FF70FEF7E7FF46F6FF00FEF7E3FF47F6DD
:10830800FF10FEF7DFFF3046FDF7ECF800F04CFAFF
:108318002846FDF72BFB0028FAD16748FFF716FC23
:1083280059A5D5E900455AA7D7E90067FFF7F6FC34
:108338000E2262496248FDF7DFF9DFF8B881DFF8FD
:10834800B891DFF864A104214846FDF7B9FFD0B918
:1083580001214846FDF7B4FF0128834613D1594A45
:10836800594B0492594A03924FF48262029203F1E4
:10837800100292E803008DE803000FCB00F064F9C7
:108388005846FDF7AFF808214846FDF799FFD0B9E0
:1083980002214846FDF794FF0128834613D1494A34
:1083A8004B4B04924B4A03924FF48262029203F1C0
:1083B800100292E803008DE803000FCB00F044F9A7
:1083C8005846FDF78FF820214046FDF779FFD0B9D0
:1083D80008214046FDF774FF0128834613D1394A26
:1083E8003D4B04923D4A03924FF48262029203F19C
:1083F800100292E803008DE803000FCB00F024F987
:108408005846FDF76FF840214046FDF759FFD0B9AF
:1084180010214046FDF754FF0128834613D1294A0D
:108428002F4B04922F4A03924FF48262029203F177
:10843800100292E803008DE803000FCB00F004F966
:108448005846FDF74FF84FF400715046FDF738FFD6
:10845800002868D14FF480515046FDF731FF0128BC
:10846800834660D141F288330393022302930023A9
:108478001D4A10A8CDE9002332463B46FFF754F9C0
:1084880003223BE0AFF3008060558FCE0000000070
:10849800A0B483EA0000000000380140001000404A
:1084A800340200208C0B002000100140001801400D
:1084B800002001400014014080040020CC05002069
:1084C8004806002092809F00A001002001E80300D8
:1084D800B8010020318D0300D001002071DE0400B6
:1084E800E8010020319A0500005A6202BC0600200B
:1084F80040070020000C0140001C0140059241F299
:10850800C2320492109A404B0392119A029203F1DC
:10851800100292E803008DE803000FCBFFF772F911
:108528005846FCF7DFFF4FF480715046FDF7C8FE50
:1085380058BB4FF480615046FDF7C2FE01288346C0
:1085480023D141F2883303930223029300232F4A55
:1085580010A8CDE9002322462B46FFF7E5F80322B1
:10856800059241F2C2320492109A294B0392119A51
:10857800029203F1100292E803008DE803000FCB8A
:10858800FFF740F95846FCF7ADFFDFF898B0DBF885
:108598000030B3F5FA7F07D94FF480411D48FDF745
:1085A8009AFE0023CBF800301B4ADFF87CB01B4949
:1085B8009368002B03DDDBF80030642B1BD840F6F2
:1085C800C4121748016891427FF6BDAE0023DFF858
:1085D8005C90DFF85CC059F8131003EB0C0202330F
:1085E8004FEA112E1C2B82F822E082F82310F2D1D8
:1085F80000230360A3E608460792069100F0C2FA3A
:10860800079A0699D4E700BF04020020005A6202C4
:108618001C02002000200140800B0020BC06002026
:10862800380400203C04002040040020CC05002031
:108638006C05002070470000024B984201D80420C6
:10864800704770477FB92A0084B02DE9F74F0CAC0A
:1086580084E80F00139BBDF8347023F07F43019327
:10866800129BDDF83880BDF83C9023F07F43109DC5
:10867800BDF844600022394600938246149CFDF7F9
:1086880025FE002249464046FDF720FE00223146DD
:108698002846FDF71BFE4FF0180B24F07F4414F416
:1086A800000218BF012249464046FDF70FFE01228D
:1086B80039465046FDF70AFE0A20FFF765FB0022FF
:1086C80039465046FDF702FE6400BBF1010B24F069
:1086D8007F44E4D1012231462846FDF7F7FD0A2000
:1086E800FFF752FB5A4631462846FDF7EFFD18249E
:1086F800009B494613F4000218BF01224046FDF7CB
:10870800E5FD012239465046FDF7E0FD0A20FFF756
:108718003BFB002239465046FDF7D8FD009B013C43
:108728004FEA430323F07F430093E1D1012231460E
:108738002846FDF7CBFD0A20FFF726FB22463146E7
:108748002846FDF7C3FD1824019B494613F400028F
:1087580018BF01224046FDF7B9FD012239465046AF
:10876800FDF7B4FD0A20FFF70FFB002239465046FB
:10877800FDF7ACFD019B013C4FEA430323F07F4327
:108788000193E1D1314601222846FDF79FFD0A20D9
:10879800FFF7FAFA22463146284603B0BDE8F04F03
:1087A80004B0FDF793BD000030B54FF48264224D4C
:1087B800224B234A87B003920495029403F11002D6
:1087C80092E803008DE803000FCBFFF73DFF01207F
:1087D800FCF788FE1B4B1C4A04950392029403F194
:1087E800100292E803008DE803000FCBFFF72CFF7F
:1087F8000120FCF777FE154B154A04950392029465
:1088080003F1100292E803008DE803000FCBFFF795
:108818001BFF0120FCF766FE0E4B0F4A04950392DE
:10882800029403F1100292E803008DE803000FCBD5
:10883800FFF70AFF07B030BD92809F00A00100201B
:1088480001E80300B8010020318D0300D0010020A9
:1088580071DE0400E8010020319A05000E4B82B059
:108868009A6942F001029A619A6902F00102009243
:10887800009ADA6942F08052DA61DB69074A03F04C
:1088880080530193019B536823F0E06343F0007326
:10889800536002B0704700BF001002400000014062
:1088A800102230B5054689B00DEB0200002100F01A
:1088B800D0FE2A682C4B9A4253D103F56C439A692F
:1088C800032442F400729A619A6904A902F40072BE
:1088D8000092009A9A69254842F010029A619A69B2
:1088E80002F010020192019A9A6942F004029A6118
:1088F8009A6902F004020292029A9A6942F0080206
:108908009A619B69059403F008030393039B0F2363
:108918000493FDF7E9FBFF2304A915480493059484
:10892800FDF7E2FB134804A904940594FDF7DCFB6A
:108938008022114C114BE2604FF4007222614FF417
:108948000062236062610023202220466360A360E6
:10895800A261E361FDF7DAF808B1FFF76BFE2C625C
:10896800656209B030BD00BF00240140001001401D
:1089780000080140000C0140FC06002008000240ED
:108988000268084B82B09A420AD103F50033DA69CB
:1089980042F01002DA61DB6903F010030193019BD6
:1089A80002B070470010004070B5064686B010222D
:1089B800002102A800F04DFE32682B4B9A4251D19B
:1089C80003F558439A6902A942F480429A619A6968
:1089D800264802F480420092009A9A69002542F0E3
:1089E80004029A619B69224C03F004030193019BE2
:1089F8004FF4007302930223039303230593FDF7B7
:108A080073FB4FF48063194802A9029303950495F8
:108A1800FDF76AFB174B204684E828008023A560F1
:108A2800E36025616561A561E561FDF76FF808B14F
:108A3800FFF700FE4FF0100C0F4B746366620F4C8B
:108A4800802284E8081000232046A360E2602361A6
:108A58006361A361E361FDF759F808B1FFF7EAFD27
:108A68003463666206B070BD0038014000080140FA
:108A78007806002058000240440002400406002006
:108A88007047FEE7FEE7FEE7FEE77047704770476E
:108A9800FCF716BD0148FDF725B900BFFC0600200C
:108AA8000148FDF71FB900BF040600200148FDF783
:108AB80019B900BF780600200148FEF75BBB00BF6C
:108AC800BC0600200148FDF7A3BF00BF40070020F7
:108AD80070B50E4615460C46A31B9D4201DC284680
:108AE80070BDAFF3008004F8010BF5E708B50A4B39
:108AF8000246196809B909491960694618680244A3
:108B08008A4206D900F070FD0C2303604FF0FF3055
:108B180008BD1A6008BD00BF44040020A01700204B
:108B28004FF0FF3070474FF4005300204B60704700
:108B380001207047002070470E4B1A6842F001026E
:108B48001A6059680C4A0A405A601A6822F08472FE
:108B580022F480321A601A6822F480221A605A6855
:108B680022F4FE025A604FF41F029A60034A044B33
:108B78009A607047001002400000FFF800400008AB
:108B880000ED00E0144A38B51068431C1360134B1D
:108B9800596803F10C040D5D114C0131B1F5806F7A
:108BA80025541446A8BF00229D68B8BF596005F136
:108BB800FF35A8BF5A609D606DB9094800F0A0FC58
:108BC80022682946064800F044FD25600120BDE8DA
:108BD8003840FCF787BC38BD48040020800B0020D3
:108BE8008007002000230F4A10B513600E4C0F4A6F
:108BF800136022680132B2F5806FB8BF1346236054
:108C0800A3680133B3F5806FA36001DBFFF7BAFFF8
:108C1800236807490122BDE8104019440548FEF7BA
:108C2800BBB900BF40040020800B0020380400209E
:108C38008C0B0020BC06002008B5C3788178C25C84
:108C48000130FEF705FC003018BF012008BD000008
:108C5800BE2310B50B4C5D212370022363705E2385
:108C6800601CA170E370FEF7D8FBEB2384F85E006C
:108C780084F85F302146BDE8104060220248FEF7C4
:108C880051B900BF6C050020BC060020BE2310B5FA
:108C98000A4C032123700423601C6370A170E370E5
:108CA800FEF7BBFBEB23A278207163712146BDE878
:108CB800104003320248FEF735B900BF4C040020CB
:108CC800BC0600200000000070B5B14D02792B7978
:108CD800A2B0934204460CD0AE4B029203F11002AC
:108CE80092E803008DE803000FCBFEF73DFB2379E4
:108CF8002B7162796B7993420CD0A74B029203F1E6
:108D0800100292E803008DE803000FCBFEF72CFB5E
:108D180063796B71A279AB7993420CD09F4B029225
:108D280003F1100292E803008DE803000FCBFEF771
:108D38001BFBA379AB71E279EB7993420CD0984B8A
:108D4800029203F1100292E803008DE803000FCBB2
:108D5800FEF70AFBE379EB71227A2B7A93420CD067
:108D6800904B029203F1100292E803008DE8030091
:108D78000FCBFEF7F9FA237A2B72627A6B7A934259
:108D88000CD0894B029203F1100292E803008DE89F
:108D980003000FCBFEF7E8FA637A6B72A27AAB7A1C
:108DA80093420CD0814B029203F1100292E8030027
:108DB8008DE803000FCBFEF7D7FAA37AAB72E27AFD
:108DC800EB7A93420CD07A4B029203F1100292E8AC
:108DD80003008DE803000FCBFEF7C6FAE37AEB72C7
:108DE800227B2B7B93420CD0724B029203F1100230
:108DF80092E803008DE803000FCBFEF7B5FA237B5A
:108E08002B73627B6B7B93420CD06B4B029203F10A
:108E1800100292E803008DE803000FCBFEF7A4FAD6
:108E2800637B6B73A27BAB7B93420CD0634B029248
:108E380003F1100292E803008DE803000FCBFEF760
:108E480093FAA37BAB73E27BEB7B93420CD05C4B36
:108E5800029203F1100292E803008DE803000FCBA1
:108E6800FEF782FAE37BEB73237C2A7C9A420FD1CC
:108E7800697C627C91420BD1A97CA27C914207D18A
:108E8800E97CE27C914203D1297D227D91421CD06C
:108E98004C4E2B743376637C7C226B7486F83430AA
:108EA800A37C06F11001AB7486F85030E37C684669
:108EB800EB7486F86C30237D2B7586F8883000F0CB
:108EC800BDFB96E80F00FEF7F3FA627D6B7D9342D7
:108ED8001DD0A37DA97D994219D06A75AB75607DB7
:108EE800A37D43EA002338485843FFF7A5FB374AD8
:108EF800374B04924FF482620390029203F11002FE
:108F080092E803008DE803000FCBFFF79DFBE37D9C
:108F1800EA7D9A421BD0207E2A7E824217D0EB75CA
:108F2800287640EA0320284B5843FFF785FB274A59
:108F3800284B04924FF482620390029203F11002CC
:108F480092E803008DE803000FCBFFF77DFB637EFB
:108F58006A7E9A4242D0A07EAA7E82423ED06B763A
:108F6800A87640EA0320184B5843FFF765FB174AD9
:108F7800194B04924FF482620390029203F110029B
:108F880092E803008DE803000FCBFFF75DFB25E0B7
:108F98006C05002008000020200000203800002078
:108FA8005000002068000020800000209800002069
:108FB800B0000020C8000020E0000020F8000020D9
:108FC80010010020E0040020A086010092809F008C
:108FD800A0010020B8010020D0010020E27EEB7E35
:108FE80093421DD0237F297F994219D0EA762B77A7
:108FF800E07E237F43EA0023C7485843FFF71CFB62
:10900800C64AC74B04924FF482620390029203F15E
:10901800100292E803008DE803000FCBFFF714FB62
:10902800627F6B7F934227D0A37FA97F994223D089
:10903800AB7741F2883303930223029300236A77C4
:10904800B84A20A8CDE90023AFA3D3E90023FEF74F
:109058006BFB0322059241F2C2320492209AB24B72
:109068000392219A029203F1100292E803008DE81C
:1090780003000FCBFEF7C6FBE27FEB7F93422AD0BB
:1090880094F8203095F82010994224D085F82030A3
:1090980041F288330393022302930023EA77A14A1B
:1090A80020A8CDE900239AA3D3E90023FEF73CFBCF
:1090B8000322059241F2C2320492209A9B4B0392FA
:1090C800219A029203F1100292E803008DE803004E
:1090D8000FCBFEF797FB94F8401095F840308B4281
:1090E80006D04020FEF794FD94F8403085F84030D3
:1090F80094F8411095F841308B4206D04120FEF794
:1091080087FD94F8413085F8413094F8421095F87D
:1091180042308B4206D04220FEF77AFD94F8423066
:1091280085F8423094F8431095F843308B4206D0C6
:109138004320FEF76DFD94F8433085F8433094F8EA
:10914800471095F847308B4206D04720FEF760FD60
:1091580094F8473085F8473094F8461095F846302B
:109168008B4206D04620FEF753FD94F8463085F82A
:10917800463094F8441095F844308B4206D0442089
:10918800FEF746FD94F8443085F8443094F84510CD
:1091980095F845308B4206D04520FEF739FD94F806
:1091A800453085F8453094F8481095F848308B429A
:1091B80036D04820FEF72CFD94F848300A2085F870
:1091C8004830FCF78FF995F84810594800F0AAFE86
:1091D80094F8483023B3574800F018FF41F2883319
:1091E80003930223029300234E4A20A8CDE90023CB
:1091F80045A3D3E90023FEF797FA0322059241F22B
:10920800C2320492209A494B0392219A029203F1A6
:10921800100292E803008DE803000FCBFEF7F2FA84
:1092280094F8491095F849308B4236D04920FEF71A
:10923800EFFC94F849300A2085F84930FCF752F9D8
:1092480095F849103A4800F06DFE94F8493023B378
:10925800384800F0DBFE41F288330393022302937F
:109268000023304A20A8CDE9002329A3D3E900230D
:10927800FEF75AFA0322059241F2C2320492209A6A
:10928800294B0392219A029203F1100292E80300FB
:109298008DE803000FCBFEF7B5FA94F84A3095F83D
:1092A8004A209A4206D085F84A3094F84A104A2053
:1092B800FEF7AEFC94F84B3095F84B209A4206D056
:1092C80085F84B3094F84B104B20FEF7A1FC1A4D53
:1092D80094F84C3095F84C209A4206D085F84C30DA
:1092E80094F84C104C20FEF793FC94F84D3095F808
:1092F8004D209A4222D085F84D3094F84D104D20DB
:10930800FEF786FC1AE000BFA0B483EA0000000064
:1093180060558FCE00000000A086010092809F005B
:10932800E8010020005A62021C020020040200200A
:10933800DBBF0008E9BF00086C05002094F84E3038
:1093480095F84E209A4206D195F84F1094F84F2080
:10935800914200F0CE8085F84E3094F84F3085F871
:109368004F30012394F8502095F85010914205D1C0
:1093780095F8510094F85110884206D085F850208D
:1093880094F8513085F85130012394F8522095F81B
:109398005210914205D195F8530094F85310884221
:1093A80006D085F8522094F8533085F853300123BD
:1093B80094F8542095F85410914205D195F8550029
:1093C80094F85510884206D085F8542094F8553002
:1093D80085F85530012394F8562095F85610914297
:1093E80005D195F8570094F85710884206D085F8AB
:1093F800562094F8573085F85730012394F85820B0
:1094080095F85810914205D195F8590094F85910DB
:10941800884206D085F8582094F8593085F8593094
:10942800012394F85A2095F85A10914205D195F8DD
:109438005B0094F85B10884206D085F85A2094F8AF
:109448005B3085F85B30012394F85C2095F85C105C
:10945800914205D195F85D0094F85D1088424AD094
:1094680085F85C2094F85D3085F85D3095F84F30CC
:1094780095F84E0043EA0020FDF724FF95F8513097
:1094880095F8500043EA0020FDF71CFF95F853308B
:1094980095F8520043EA0020FDF714FF95F855307F
:1094A80095F8540043EA0020FDF70CFF95F8573073
:1094B80095F8560043EA0020FDF704FF95F8593067
:1094C80095F8580043EA0020FDF7FCFE95F85B305C
:1094D80095F85A0043EA0020FDF7F4FE95F85C0081
:1094E80095F85D3043EA002022B0BDE87040FDF7F2
:1094F800E9BE002336E7002BB8D122B070BD00BF0B
:1095080070B504464678FFF797FB054648B9A27838
:1095180040F6B833033221461A48FDF7A7FC28461F
:1095280070BD032EFBD8DFE806F0022026290023B1
:10953800154EA2785D1C0532DBB29A420FDA134849
:1095480000F064FDBFF34F8F1149124BCA6802F453
:10955800E0621343CB60BFF34F8F00BFFDE7E15CD0
:10956800304600F0DFFC2B46E3E72046FFF7ACFB74
:10957800FFF78CFBD3E7FFF76BFBD0E70648FEF756
:10958800E1FACCE7BC060020C7BF0008CDBF000841
:1095980000ED00E00400FA056C050020002103E05E
:1095A8000B4B5B58435004310A480B4B42189A4204
:1095B800F6D30A4A02E0002342F8043B084B9A42D9
:1095C800F9D3FFF7B9FA00F015F8FEF729FC704750
:1095D800D0C2000800000020040400200804002075
:1095E800A0170020FEE70000014B1868704700BF75
:1095F8003402002070B500250C4E0D4CA41BA4109D
:10960800A54209D102F08AFC00250A4E0A4CA41B87
:10961800A410A54205D170BD56F8253098470135EC
:10962800EEE756F8253098470135F2E7C8C200083A
:10963800C8C20008C8C20008CCC2000810B5431E42
:109648000A44914200D110BD11F8014B03F8014FB3
:10965800F7E703460244934200D1704703F8011B21
:10966800F9E7002B2DE9F0471E46BBBF03F1004385
:109678001E4600232D2388B0149F129927F0200737
:10968800462F1446109DDDF84CA00B7004D0452FD2
:1096980000D10135022300E0032307AA049206AA99
:1096A80003928DE828042246334600F0B9FE472F7E
:1096B800804602D1119BDB0726D5462F08EB05090A
:1096C80011D198F80030302B0AD10022002320460F
:1096D8003146FBF7D9F918B9C5F10105CAF80050A8
:1096E800DAF8003099440022002320463146FBF77F
:1096F800CBF938B93022079B994505D9591C0791F0
:109708001A70F8E7CDF81C904046079B159AA3EB12
:109718000803136008B0BDE8F0870346F7B50029D1
:1097280003F8022BB6BF2D222B2249420929427089
:1097380021DD0DF1070217460A2691FBF6F506FB17
:109748001511092D01F1300102F8011C02F1FF3455
:10975800294609DC3031023A04F8011CBA421C4699
:1097680004D3201A03B0F0BD2246E6E712F8011B25
:1097780003F8011BF2E730221C46114404F8022BBF
:109788005970EEE72DE9F04F91B00C461A9F9346B9
:109798001E46054601F094FD036818460993FAF73A
:1097A8003FFD00230E933B680A90073323F007031D
:1097B80003F1080294F81880D4F800A03A60D3E9BD
:1097C8000023C4E91223D4F84C90A76C29F0004375
:1097D8000B934FF0FF32A64B38460B99FBF786F9EF
:1097E800002840F0F7814FF0FF32A14B38460B9923
:1097F800FBF75EF9002840F0ED810022002338468F
:109808004946FBF74BF910B12D2384F84330994BA7
:10981800994FB8F1470F98BF1F4603234FF000092F
:1098280023612AF00403236000965B460FAA2146B1
:10983800284600F0DFF9013040F09A804FF0FF3001
:1098480011B0BDE8F08F62680EA8531C0DF1340EFC
:109858004AF4806341D106226260002123600193AB
:1098680063680DF133020590029200933A464B4625
:109878000691CDF81080CDF80CE02846FFF7F1FEF0
:1098880008F0DF03472B074609D10D9BD81C02DBE4
:109898006268934259DDA8F102085FFA88F8B8F1C6
:1098A800650F0D9936D80139424604F150000D91E3
:1098B800FFF733FF0E9A81468318012A236102DCE1
:1098C8002268D10701D5013323619DF83330002B7D
:1098D800AAD02D2384F84330A6E7B8F1670F02D049
:1098E800B8F1470FB9D19AB1002106910DF13301B2
:1098F8008DE80C00236005903A46CDF81080CDF82D
:109908000CE002914B462846FFF7ABFE0746BCE742
:109918000122A1E7B8F1660F19D1002963680CDDAF
:10992800216113B92268D20702D501330B442361A0
:109938000D9B4FF00009A365C7E713B92268D0074C
:1099480001D50233F3E70123F1E74FF067080D9BD8
:109958000E9A934205DB22682361D107E8D50133CB
:10996800E5E7002BCCBF0123C3F102031344DEE774
:1099780023685A0507D423693A4659462846B0470A
:1099880001302AD15AE7B8F1650F40F2DC80D4E9FA
:10999800120100220023FBF777F8002839D00123B1
:1099A800364A59462846B04701303FF447AF0E9B28
:1099B8000D9A9A4202DB2368D8070ED50A9B099AAA
:1099C80059462846B04701303FF438AF002704F124
:1099D8001A080E9B013B9F4211DB23689F0708D59D
:1099E800002704F11908E3680F9A9B1A9F42C0F2F6
:1099F800E780E0680F9B9842B8BF184620E701232C
:109A0800424659462846B04701303FF417AF013760
:109A1800DFE70D9B002B33DC0123184A5946284603
:109A2800B04701303FF40AAF0D9B23B90E9B13B921
:109A38002368D907D1D50A9B099A59462846B047C1
:109A480001303FF4FBAE4FF0000804F11A090D9BFA
:109A58005B42984501DB0E9B8EE701234A46594637
:109A68002846B04701303FF4E9AE08F10108EEE7B7
:109A7800FFFFEF7F04C0000808C0000814C00008FA
:109A88000E9AA36D9A42A8BF1A46002A904636DC61
:109A98004FF0000A04F11A0328EAE8780B93D4F887
:109AA8005890A9EB08039A4531DB0E9B0D9A9A4210
:109AB80038DB2368DA0735D40E9B0D99A3EB09022E
:109AC800A3EB01089045A8BF9046B8F1000F31DC20
:109AD800002728EAE87804F11A090D9A0E9B9B1AC8
:109AE800A3EB08039F42BFF678AF01234A465946C5
:109AF8002846B04701303FF4A1AE0137EDE71346E1
:109B080059463A462846B0470130C1D196E6012366
:109B18000B9A59462846B04701303FF48FAE0AF1F8
:109B2800010ABCE70A9B099A59462846B047013002
:109B3800C2D183E6434607EB090259462846B04797
:109B48000130C5D17AE60E9A012A01DCDB0734D54B
:109B580001233A4659462846B04701303FF46EAED5
:109B68000A9B099A59462846B04701303FF466AE29
:109B7800D4E9120100220023FAF786FF50B100272A
:109B880004F11A080E9B013B9F420CDB4B4604F183
:109B98005002F2E60E9B7A1C013B59462846B04714
:109BA8000130F3D14AE60123424659462846B047D8
:109BB80001303FF443AE0137E4E701233A46ECE7CE
:109BC8000123424659462846B04701303FF436AE95
:109BD800013708E73A464B4638464946FAF786FFC2
:109BE80000283FF430AE014B014F12E60CC00008CC
:109BF80010C000082DE9F04791461F468A680B6996
:109C080006469342B8BF1346C9F8003091F843207E
:109C18000C46DDF8208012B10133C9F80030236802
:109C2800990642BFD9F800300233C9F800302568D8
:109C380015F0060507D104F1190AE368D9F80020E0
:109C48009B1A9D422ADB94F843302268003318BFE0
:109C5800012392062FD404F1430239463046C04707
:109C6800013022D02368E56803F00603042B18BFEF
:109C78000025D9F800204FF0000908BFAD1AA368E5
:109C8800226908BF25EAE5759342C4BF9B1AED18FF
:109C98001A344D451BD10020BDE8F08701235246F8
:109CA80039463046C047013003D14FF0FF30BDE898
:109CB800F0870135C1E73020E11881F843005A1CCC
:109CC80094F845102244023382F84310C3E7012375
:109CD800224639463046C0470130E6D009F101092D
:109CE800D7E700002DE9F04317460A7E85B06E2AB3
:109CF800984606460C460C9B01F1430E00F0BC80CA
:109D08001AD8632A2ED00AD8002A00F0C880582A08
:109D180000F08A8004F1420584F842202AE0642A8F
:109D280001D0692AF6D121681A6811F0800F23D072
:109D3800111D1960136827E0732A00F0B48008D851
:109D48006F2A2AD0702AE5D10A6842F020020A60F8
:109D580003E0752A21D0782ADCD178226F4984F86B
:109D6800452064E01A6801F14205111D1960136865
:109D780084F842300123A3E011F0400F02F10401FE
:109D88001960D7D0B2F90030002B03DA2D225B42DC
:109D980084F8432062490A2217E02068196810F005
:109DA800800F03D0081D18600B6806E010F0400F04
:109DB80001F104001860F7D00B886F2A14BF0A223B
:109DC80008225749002084F843006568002DA560E3
:109DD800C0F29C80206820F004002060002B3FD156
:109DE800002D40F095807546082A0BD12368DA07C4
:109DF80008D5236962689A42DEBF302305F8013C22
:109E080005F1FF35AEEB05032361CDF800803B4635
:109E180003AA21463046FFF7EDFE013055D14FF039
:109E2800FF3005B0BDE8F08381F845203C49226841
:109E3800186812F0800F00F104051D6001D0036856
:109E480002E05506FBD50388D00744BF42F0200244
:109E580022601BB9226822F0200222601022B1E79A
:109E68007546B3FBF2F002FB1033CB5C05F8013DFD
:109E780003460028F5D1B7E708681A6810F0800F84
:109E8800496904D0101D18601368196007E010F0C4
:109E9800400F02F1040018601368F6D019800023FF
:109EA80075462361B1E71A68111D1960156800210C
:109EB8006268284601F07EFA08B1401B606063685A
:109EC8002361002384F843309FE723692A463946F3
:109ED8003046C0470130A2D023689B0707D500252C
:109EE80004F11909E368039A9B1A9D4205DBE068AF
:109EF800039B9842B8BF184693E701234A46394660
:109F08003046C04701308AD00135EBE7002BA7D196
:109F18000B7804F1420584F8423065E727C0000851
:109F280016C000080FB40A4B13B51C6824B1A36906
:109F380013B9204601F03AF905AB049AA168204606
:109F4800019301F0F7FD02B0BDE8104004B070477E
:109F58003402002070B50E46054618B183690BB966
:109F680001F024F9AB69AC6813B9284601F01EF971
:109F7800234B9C4217D16C68A3891B071DD5236905
:109F8800DBB1013EA36816F8011F013BA360E9B9E4
:109F9800002B2EDA22460A21284600F0F5F8013077
:109FA80011D00A2070BD174B9C4201D1AC68E3E781
:109FB800154B9C4208BFEC68DEE72146284600F0B6
:109FC80035F90028DDD04FF0FF3070BD002B04DAE2
:109FD800A269934206DB0A2904D023685A1C22602E
:109FE8001970CFE72246284600F0CEF80130C9D1D3
:109FF800E9E70A2023685A1C2260187070BD00BF68
:10A0080068C0000888C0000848C00008024B014624
:10A018001868FFF79FBF00BF3402002000294FF4E3
:10A0280080630CBF0222002200F000B82DE9F7433C
:10A038001D46514B04461E680F46904626B1B3692B
:10A0480013B9304601F0B2F84C4B9C4252D17468B7
:10A05800B8F1020F06D0B8F1010F00F28980002D87
:10A06800C0F286802146304601F036F8616B41B176
:10A0780004F14403994202D0304601F089FC0023E0
:10A0880063630023A3616360A3891B0603D5216969
:10A09800304601F07DFCA389B8F1020F23F44A632E
:10A0A80023F00303A3815DD001AB6A462146304605
:10A0B80001F014F9A3891843A0812DBB009D2846FF
:10A0C80001F070F9074600284ED1DDF80090A94547
:10A0D8003CD14FF0FF30A38943F00203A381002352
:10A0E800A36004F14703236023610123636103B084
:10A0F800BDE8F083224B9C4201D1B468A8E7214B0C
:10A108009C4208BFF468A3E7002FD8D0B36913B9FD
:10A11800304601F04BF8B8F1010F08BFA38927605A
:10A1280004BF43F00103A381A389276113F008004A
:10A1380065611BD013F001004FF000031FBF6D4293
:10A14800A360A561184608BFA560D0E7484601F09E
:10A1580029F907460028BCD0A3894D4643F080035F
:10A16800A381D3E70020B6E7A946F5E7A060BEE7DC
:10A178004FF0FF30BBE700BF3402002068C0000882
:10A1880088C0000848C00008F8B50E4614460546C1
:10A1980018B183690BB901F009F8214B9C422AD107
:10A1A8006C68A369A360A3891A072ED5236963B3D2
:10A1B80023692068F6B2C01A63693746984204DBFF
:10A1C8002146284600F088FF28BBA3680130013BE0
:10A1D800A36023685A1C22601E706369984204D0E9
:10A1E800A389DB0719D50A2E17D12146284600F086
:10A1F80073FF90B10FE00B4B9C4201D1AC68D0E7E4
:10A20800094B9C4208BFEC68CBE72146284600F082
:10A218000DF80028CCD04FF0FF373846F8BD00BF06
:10A2280068C0000888C0000848C00008324B70B5F4
:10A238001D6806460C4625B1AB6913B9284600F0DF
:10A24800B5FF2E4B9C420FD16C68B4F90C309AB212
:10A2580015072CD4D00611D40922326043F04003EC
:10A26800A3814FF0FF3070BD254B9C4201D1AC68F3
:10A27800EBE7244B9C4208BFEC68E6E7510712D590
:10A28800616B41B104F14403994202D0304601F0B8
:10A298007FFB00236363A38923F02403A3810023A6
:10A2A800636023692360A38943F00803A3812369BA
:10A2B8004BB9A38903F42073B3F5007F03D021467B
:10A2C800304601F02FF8A28912F001030CD00023C8
:10A2D800A36063695B42A361236953B9B4F90C3085
:10A2E80013F08000BAD170BD920758BF6369A360AC
:10A2F800F2E70020F7E700BF3402002068C000083A
:10A3080088C0000848C000082DE9F74F03690C69A8
:10A3180080469C4200F38280013C01F1140700F161
:10A32800140657F8245056F824000135B0FBF5F50B
:10A338004FEA840E06EB0E0307EB0E0901938DB36B
:10A348004FF0000A3846B446D34650F8042B93B26F
:10A3580005FB03A3120C4FEA134A05FB02A29BB2AA
:10A36800ABEB0303BCF800B04FEA124A5B441FFA98
:10A3780082FBDCF800208145CBEB124202EB234242
:10A388009BB243EA02434FEA224B4CF8043BDCD22F
:10A3980056F80E3033B9019B043B9E421A4631D31E
:10A3A800C8F81040404601F01CFA002826DB304669
:10A3B8004FF0000E013557F8041BD0F800C08BB2DF
:10A3C800AEEB03031FFA8CF213440A0CC2EB1C42D7
:10A3D80002EB23429BB243EA0243B9454FEA224EBD
:10A3E80040F8043BE7D256F8242006EB84032AB948
:10A3F800043B9E421A460BD3C8F81040284603B0C7
:10A40800BDE8F08F1268043B002AC9D1013CC4E7BB
:10A418001268043B002AEFD1013CEAE70020EEE78E
:10A428002DE9F04F466A95B00446219DCDE90223F7
:10A438003EB9102000F0B6FF606246608660066094
:10A44800C660636A196851B15A68012393404A602B
:10A458008B60204600F0F0FF0022636A1A60039BBD
:10A46800002BB7BF012300232B60039BAEBF2B60DB
:10A4780023F000430393DDF80C90AB4B33EA090358
:10A488001BD142F20F73209A1360029B23B9C9F3C0
:10A498001300002800F08385229B53B9A34B21E0C9
:10A4A800A34B06930833229A1360069815B0BDE8AB
:10A4B800F08F9E4B06930333F5E7DDE90267002230
:10A4C800002330463946FAF7DFFA804660B10123A7
:10A4D800209A1360229B002B00F05E85954B229AF0
:10A4E8001360013B0693E0E712AB019313AB0093B3
:10A4F80032463B46204601F0EDF9C9F30A5582463B
:10A50800002D7DD03046C7F3130343F07F5141F44B
:10A518004011A5F2FF35CDF840800022864BF9F7AF
:10A5280097FE7BA3D3E90023FAF746F87AA3D3E989
:10A538000023F9F78FFE064628460F46F9F7D6FF9F
:10A5480077A3D3E90023FAF737F802460B463046DB
:10A558003946F9F77FFE06460F46FAF7DDFA00227C
:10A568008346002330463946FAF798FA58B15846D8
:10A57800F9F7BCFF02460B4630463946FAF784FA2B
:10A5880008B90BF1FF3BBBF1160F58D8DDE90223E0
:10A598006A4901EBCB01D1E90001FAF79DFA0028DD
:10A5A8004FD000230BF1FF3B0D93129B5D1B6B1EDD
:10A5B800079343BF0023C5F1010807934FF0000834
:10A5C800BBF1000F3FDB079BCDF830B05B4407932E
:10A5D800002308931E9B092B00F2B480052BC4BFEF
:10A5E800043B1E931E9BC8BF0026A3F10203D8BFDD
:10A5F8000126032B00F2B280DFE803F084862D7871
:10A60800139B129D1D4405F23243202B11DD029A43
:10A6180005F21240C3F1400322FA00F009FA03F3ED
:10A628001843F9F753FF0123A1F1F871013D109385
:10A6380073E7C3F12000029B03FA00F0F1E701235E
:10A64800B2E70D90B1E7CBF1000308930023A8EB24
:10A658000B080C93BEE7012309931F9B002B40F3C3
:10A6680080809946049300220421656A6A6001F19A
:10A6780014029A427AD96968204600F0A9FE636AF2
:10A6880028601B68B9F10E0F069300F2F080002EC7
:10A6980000F0ED80DDE90223BBF1000FCDE90E23C8
:10A6A80079DD264A0BF00F034FEA2B1602EBC303A2
:10A6B800F006D3E90023CDE90A235CD5DDE90E01D4
:10A6C8001F4B0325D3E90823FAF7A0F8CDE90201C7
:10A6D80006F00F061A4F002E4FD1DDE90A23DDE9F7
:10A6E8000201FAF793F8CDE902016EE0012309931C
:10A6F8001F9B5B4403F1010904934B46012BB8BF30
:10A708000123B0E70023A7E70023F0E7AFF30080B9
:10A7180061436F63A787D23FB3C8608B288AC63F5F
:10A72800FB799F501344D33F0000F07F41C00008DD
:10A7380038C0000815C000080000F83FD0C0000865
:10A74800A8C000080126002309961E934FF0FF3386
:10A7580000220493994612231F9284E70123099348
:10A76800F4E70123049399461A46F5E76A68490015
:10A7780001326A607BE70225ACE7F10708D5DDE91D
:10A788000A01D7E90023F9F717FFCDE90A010135D6
:10A79800761008379FE700F0A580DDE90E01CBF1C0
:10A7A8000006A24B06F00F0203EBC203D3E9002315
:10A7B800F9F702FF02250023CDE902019C4F36116B
:10A7C800002E40F08480002B8DD10D9B002B00F0D3
:10A7D8008B80DDE90223CDE90A23DDE90A010022A5
:10A7E800944BFAF75BF900287ED0B9F1000F7BD0C3
:10A7F800049B002B37DDDDE90A0100228E4BF9F7B7
:10A80800DBFECDE90201049E0BF1FF370135284636
:10A81800F9F76CFEDDE90223F9F7CEFE874B00223B
:10A82800F9F718FDCDE90A010B9BA3F150750B95BB
:10A83800002E5CD1DDE902010022814BF9F708FD09
:10A848000A9A2B46CDE90201FAF746F9002840F0AA
:10A85800F782DDE902010A9A05F10043FAF71EF9C9
:10A86800002840F0EB82DDE90E23CDE90223139B9B
:10A87800002BC0F25081BBF10E0F00F34C816B4BE3
:10A8880003EBCB03D3E90023CDE904231F9B002B63
:10A8980080F2DA80B9F1000F00F3D68040F0CD8263
:10A8A800DDE904010022664BF9F786FEDDE90223A3
:10A8B800FAF708F94E464F46002840F0A482069B56
:10A8C800069A5D1C31230BF1010B13709FE2F2070E
:10A8D80005D5D7E90023F9F76FFE01230135761076
:10A8E80008376DE7022570E75F464E468FE7069A00
:10A8F8004E4B32441192099A711E002A48D003EB3C
:10A90800C103D3E9002300204E49F9F77FFFDDE9B1
:10A918000A23F9F79DFCCDE90A01069DDDE902014C
:10A92800FAF7FAF80646F9F7E1FD02460B46DDE9C3
:10A938000201F9F78DFCDDE90A23303605F8016BD1
:10A94800CDE90201FAF7AAF8002864D1DDE902236B
:10A9580000203849F9F77CFCDDE90A23FAF79EF86C
:10A96800002840F0B980119B9D423FF47CAFDDE99F
:10A978000A010022304BF9F71FFE0022CDE90A0137
:10A98800DDE902012C4BF9F717FECDE90201C5E715
:10A9980003EBC101D1E90001DDE90A23F9F70CFE57
:10A9A800CDE90A01069DDDE90201FAF7B5F8064688
:10A9B800F9F79CFD02460B46DDE90201F9F748FC70
:10A9C8003036119B05F8016BAB42CDE902014FF01F
:10A9D800000224D11B4BDDE90A01F9F73BFC0246D2
:10A9E8000B46DDE90201FAF777F8002874D1DDE9B2
:10A9F8000A2300201349F9F72BFC02460B46DDE930
:10AA08000201FAF74BF800283FF42DAF15F8013C86
:10AA18006A1E302B01D0BB464DE01546F6E7064BC3
:10AA2800F9F7CAFDCDE90201BDE700BFD0C00008B3
:10AA3800A8C000080000F03F0000244000001C40AF
:10AA4800000014400000E03F069DDDE90267DDE9F3
:10AA5800042330463946F9F7D9FEFAF75DF88046FF
:10AA6800F9F744FDDDE90423F9F7A6FD02460B4694
:10AA780030463946F9F7ECFB08F1300605F8016B6A
:10AA8800069E0246AE1BB1450B4637D1F9F7E2FBED
:10AA980006460F4602460B46DDE90401F9F7FEFFBC
:10AAA800C8B9DDE9040132463B46F9F7EDFF10B1BC
:10AAB80018F0010F0FD15146204600F0BDFC0023CD
:10AAC800209A2B700BF101031360229B002B3FF49B
:10AAD800ECAC1D60E9E45F4615F8012C6B1E392AC1
:10AAE80006D1069A9A4207D13023137013460137CC
:10AAF8001A7801321A708EE71D46EDE70022B54B31
:10AB0800F9F75AFD0022002306460F46F9F7BCFF65
:10AB180000289CD0CFE7099A002A00F029811E9AC4
:10AB2800012A00F30E81109A002A00F0068103F230
:10AB380033434546089E079A01211A442046984403
:10AB4800079200F019FD0746002D0BDD079B002B2F
:10AB580008DDAB42A8BF2B46079AA8EB0308ED1AFD
:10AB6800D31A0793089BFBB1099B002B00F00481C3
:10AB7800002E11DD39463246204600F093FD52463C
:10AB880001460746204600F000FD51460A9020463F
:10AB980000F052FC0A9B9A46089B9A1B04D0514627
:10ABA800204600F07FFD82460121204600F0E4FCAB
:10ABB8000C9B0646002B40F3E1801A4601462046CE
:10ABC80000F070FD1E9B0646012B40F3DA8000233F
:10ABD8000893336906EB8303186900F07FFCC0F122
:10ABE8002000079B184410F01F0000F0F080C0F10F
:10ABF8002003042B40F3E280079BC0F11C00804433
:10AC0800054403440793B8F1000F05DD5146424659
:10AC1800204600F095FD8246079B002B05DD314656
:10AC28001A46204600F08CFD06460D9B002B00F0CE
:10AC3800D3803146504600F0D4FD002880F2CC8005
:10AC4800002351460A22204600F00DFC099B0BF117
:10AC5800FF3B8246002B00F0A981002339460A22D7
:10AC6800204600F000FC049B0746002B03DC1E9BDB
:10AC7800022B00F3B980002D05DD39462A4620460F
:10AC880000F05EFD0746089B002B00F010817968F4
:10AC9800204600F09DFB05463A6907F10C01023297
:10ACA80092000C30FEF7CAFC01222946204600F02B
:10ACB80047FD07970746029BDDF8188003F001035C
:10ACC800089331465046FFF71FFB0799054600F1E8
:10ACD8003009504600F085FD3A460290314620463C
:10ACE80000F099FDC3680246002B40F0E28001465F
:10ACF8000990504600F075FD0346099A1146204612
:10AD0800099300F099FB099B002B40F0D4801E9A10
:10AD1800002A40F0D080089A002A40F0CC80B9F18F
:10AD2800390F00F0E880029B002B01DD05F13109A5
:10AD380008F1010588F800906BE0129BC3F1360317
:10AD4800F7E6089B09F1FF36B342B7BF089B9E1B85
:10AD5800F21A0C9BBFBF08969B180C930026B9F1FA
:10AD6800000FB9BFA8EB0905002345464B46E2E6AC
:10AD7800089E4546099FE7E6089A10E71E9B012BA7
:10AD880018DC029BB3B9039BC3F31303A3B9039B5A
:10AD980023F000431B0D1B052BB1079B08F101088D
:10ADA80001330793012308930C9B002B7FF411AF09
:10ADB800012016E70023F6E7029BF4E73FF423AFF0
:10ADC800079A1C331A4498441D4413461AE703464D
:10ADD800F6E700BF00002440B9F1000F33DC1E9BEA
:10ADE800022B30DDCDF81090049B63B93146052263
:10ADF800204600F038FB01460646504600F0F1FCBC
:10AE080000283FF75CAD1F9B069D6FEA030B0023EC
:10AE180007933146204600F00FFB002F3FF44BAE5E
:10AE2800079B2BB1BB4203D01946204600F004FB18
:10AE38003946204600F000FB3DE600263746E2E7AB
:10AE4800BB4637463BE5099BCDF81090002B7FF4B5
:10AE580012AF069D31465046FFF756FA069B00F1A1
:10AE6800300905F8019B049AEB1A9A4200F3818095
:10AE7800069B012AACBF9B18013398460023079311
:10AE880051460122204600F05BFC3146824600F024
:10AE9800A8FC002834DC02D119F0010F30D1454656
:10AEA80015F8013C6A1E302BB3D11546F8E7384631
:10AEB800FFE6012322E7029A002A04DB28D11E9A22
:10AEC80032BB089A22BB002B7FF732AF51460122D2
:10AED800204600F035FC3146824600F082FC00280E
:10AEE80005DC7FF425AF19F0010F3FF421AFB9F16C
:10AEF800390F7FF41BAF392308F1010808F8013C2A
:10AF0800454615F8013C6A1E392B3AD001333FE01B
:10AF1800002B08F1010505DDB9F1390FEBD009F176
:10AF2800010907E7069B049AEB1A9342A84605F81D
:10AF3800019CA5D0514600230A22204600F093FA2E
:10AF4800079B8246BB424FF00A024FF00003079965
:10AF5800204604D100F087FA07900746B1E600F0D2
:10AF680082FA002307900A223946204600F07BFA2D
:10AF7800F3E7514600230A22204600F074FA82467D
:10AF880068E7069B934205D13123069A0BF1010B22
:10AF980013703EE71546B4E7094BFFF7A3BA229BA7
:10AFA800002B7FF47DAA074BFFF79CBA049B002B6C
:10AFB8003FF74FAF1E9B022B7FF74BAF14E700BF45
:10AFC80014C0000838C000088A892DE9F0410546F8
:10AFD80010070C465AD44B68002B05DC0B6C002B71
:10AFE80002DC0020BDE8F081E66A002EF9D00023DB
:10AFF80012F480522F682B6033D0606DA3895A07F2
:10B0080005D56368C01A636B0BB1236CC01A0023A3
:10B018000246E66A216A2846B047431CA38906D13E
:10B0280029681D294BD82B4ACA40D60747D5002284
:10B0380062602269D904226004D5421C01D12B68C0
:10B0480003B96065616B2F600029CAD004F144031D
:10B05800994202D0284600F09BFC00206063BDE8BE
:10B06800F081216A01232846B047411CC6D12B68CC
:10B07800002BC3D01D2B01D0162B01D12F60B0E7B8
:10B08800A38943F04003A381BDE8F0810F69002F35
:10B09800A7D0930718BF00230E6808BF4B69A6EB1B
:10B0A80007080F608B60B8F1000F9ADD43463A46F7
:10B0B800216A2846A66AB047002807DCA38943F01E
:10B0C8004003A3814FF0FF30BDE8F0810744A8EBAF
:10B0D8000008E8E70100402038B50B6905460C4632
:10B0E800DBB118B183690BB900F060F80C4B9C42D6
:10B0F80009D16C68B4F90C307BB121462846BDE80B
:10B108003840FFF761BF074B9C4201D1AC68F1E7BB
:10B11800054B9C4208BFEC68ECE7002038BD00BF37
:10B1280068C0000888C0000848C00008014900F04D
:10B13800A9B800BFE1B00008002310B504460360B9
:10B148004360836081814366C28103614361836197
:10B15800194608225C30FEF77CFA054B24626362CC
:10B16800044BA362044BE362044B236310BD00BF8E
:10B1780089BD0008ABBD0008E3BD000807BE000894
:10B1880070B568254A1E55430E4605F1740100F056
:10B198004BFC044640B1002180E842000C30A0601E
:10B1A80005F16802FEF755FA204670BD836910B5AF
:10B1B800044633BB8364C3640365124B124A1B689D
:10B1C8008262984204BF0123836100F01FF8606027
:10B1D800204600F01BF8A060204600F017F8002277
:10B1E800E06004216068FFF7A7FF01220921A06839
:10B1F800FFF7A2FF02221221E068FFF79DFF01235B
:10B20800A36110BD00C0000835B10008F8B51C4B9B
:10B2180007461E68B36913B93046FFF7C7FF4836BB
:10B22800B4687368013B03D5336833B13668F7E710
:10B23800B4F90C506DB16834F4E704213846FFF7CF
:10B248009FFF30600028F1D10C2304463B60204664
:10B25800F8BD4FF6FF73E38101236566A38125607E
:10B26800A560656025616561A5610822294604F12C
:10B278005C00FEF7EEF96563A563A564E564E6E79F
:10B2880000C000082DE9F84380468946002600F1F1
:10B29800480414B93046BDE8F883A5686768013FDB
:10B2A80001D52468F5E7AB89012B07D9B5F90E302C
:10B2B800013303D029464046C84706436835EEE7C0
:10B2C800044B1B68186A044B002808BF1846F03066
:10B2D800704700BF340200209802002070B50E4667
:10B2E800B1F90E1090B0002914461D4607DA002364
:10B2F8002B60B3891A0610D44FF480630EE001AABC
:10B3080000F0A4FD0028F2DB029A02F47042A2F5D4
:10B3180000535A425A412A60EEE740230020236036
:10B3280010B070BD8B8973B59D0706460C4607D5CE
:10B3380004F14703236023610123636102B070BDF8
:10B3480001AB6A46FFF7CAFF00990546304600F090
:10B358006BFB48B9B4F90C309A05EFD423F003031A
:10B3680043F00203A381E3E70D4BB362A389206096
:10B3780043F08003A381009B20616361019B5BB163
:10B38800B4F90E10304600F073FD28B1A38923F0FC
:10B39800030343F00103A381A3891D43A581CDE7DE
:10B3A80035B10008024B0146186800F03DBB00BFEC
:10B3B8003402002010B5C9B202449042034601D1BC
:10B3C800002010BD1C7801308C42F6D1184610BD03
:10B3D80070B5456A04460E463DB91020FFF7E2FFF6
:10B3E8006062456085600560C560656AEB6883B129
:10B3F800636ADB6853F82600B8B9012101FA06F53B
:10B408006A1D9200204600F0B4FA60B1466085607B
:10B418000EE021220421204600F0ABFA636AE860BE
:10B42800DB68002BE4D1002070BD026843F82620B9
:10B4380000230361C36070BD70B5446A06460D46BB
:10B448003CB91020FFF7AEFF70624460846004606E
:10B45800C4603DB1736A6A68DB6853F822102960DA
:10B4680043F8225070BD2DE9F0411F4606460C46B0
:10B4780000230D6901F1140EDEF80000013381B2DA
:10B4880002FB0171000C0F0C02FB007089B201EB8A
:10B4980000419D424FEA10474EF8041BECDCD7B13F
:10B4A800A3689D4212DB616830460131FFF790FFC7
:10B4B8008046226904F10C01023292000C30FEF73A
:10B4C800BDF821463046FFF7B7FF444604EB850335
:10B4D80001355F6125612046BDE8F081020C120448
:10B4E8000346B2B90304102013F07F4F04BF1B02B8
:10B4F800083013F0704F04BF1B01043013F0404FA5
:10B5080004BF9B000230002B06DB5B0003D5013033
:10B5180070470020E8E7202070470368014613F0D1
:10B5280007020BD0DA0723D4980749BF5B089B08AA
:10B5380001200B605CBF0B600220704798B2A8B96D
:10B5480010201B0C13F0FF0F04BF1B0A08301A074A
:10B5580004BF1B0904309A0704BF9B080230DA07AE
:10B5680002D45B0806D001300B6070471046E9E74B
:10B57800002070472020704710B50C460121FFF7C6
:10B5880027FF01224461026110BD2DE9F74F1446DF
:10B598000A69236989469A42BEBF0B46A1461C46E2
:10B5A800D9F81070D4F810A0D9F80830D9F80410D8
:10B5B80007EB0A069E42C8BF0131FFF709FF00F1F9
:10B5C80014052B46002205EB8608434516D304F1E3
:10B5D800140209F1140102EB8A0301EB87070193B6
:10B5E800019C134694420CD8002E03DD58F8043D04
:10B5F800002B54D0066103B0BDE8F08F43F8042B4C
:10B60800E3E7B3F800A00432BAF1000F20D0AE4649
:10B6180089464FF0000C59F8044BBEF800B0A3B2AD
:10B628000AFB03B34FEA144BDEF8004063444FEAC9
:10B63800144C0AFB0BC404EB13449BB243EA0443C7
:10B648004F454FEA144C4EF8043BE4D8CEF800C0FE
:10B6580032F8029CB9F1000F1FD0AE468C464FF06D
:10B66800000A2B68BCF80040BEF802B09BB209FB88
:10B6780004B4A24443EA0A434EF8043B5CF8043B92
:10B68800BEF800401B0C09FB0343674503EB1A4354
:10B698004FEA134AE6D8CEF800300435A0E7013E59
:10B6A800A2E700002DE9F843154612F0030206460A
:10B6B8000F4607D0214C013A002354F82220FFF707
:10B6C800D2FE0746AD1035D0746A3CB91020FFF79A
:10B6D80069FE7062446084600460C460D6F82480A7
:10B6E800D8F808404CB940F271213046FFF744FFC2
:10B6F80000230446C8F8080003604FF00008EB0771
:10B708000AD5394622463046FFF73FFF814639467B
:10B718003046FFF791FE4F466D100BD0206838B9C0
:10B72800224621463046FFF730FF2060C0F80080EF
:10B738000446E4E73846BDE8F88300BF98C100082E
:10B748002DE9F0470C460746164623694FEA621A68
:10B758000AEB03094968A36809F10105AB4231DB2B
:10B768003846FFF735FE00228046114600F11403E3
:10B7780052452ADB20692AEAEA7A04F1140116F014
:10B788001F0203EB8A0301EB800E22D00020C2F1D6
:10B79800200C0E689640304343F8040B51F8040B14
:10B7A8008E4520FA0CF0F4D8186008B109F10205AA
:10B7B800013D3846C8F810502146FFF73DFE404687
:10B7C800BDE8F08701315B00C8E743F82210013279
:10B7D800CEE7043B51F8042B8E4543F8042FF9D8E3
:10B7E800E6E703690A6930B59B1A0CD19200143058
:10B7F80014318418114454F8045D51F8042D95420D
:10B8080003D005D30123184630BDA042F3D3FAE78D
:10B818004FF0FF33F7E72DE9F0470D46074611468D
:10B8280028461446FFF7DDFF061E08D13146384684
:10B83800FFF7CEFD012346610361BDE8F087A4BF91
:10B8480023462C4638466168A6BF1D4600260126B9
:10B85800FFF7BEFD4FF0000CC6602B69266904F1A6
:10B86800140205F1140902EB860709EB830800F1BD
:10B87800140152F804AB59F8045B1FFA8AF36344C5
:10B88800ACB21B1B2C0CC4EB1A4404EB23449BB234
:10B898004FEA244CC84543EA0444964641F8044B11
:10B8A800E7D8BE4505D351F8043D8BB10661BDE824
:10B8B800F0875EF8044BA2B26244131403EB1443FE
:10B8C80092B242EA03424FEA234C41F8042BE8E7DC
:10B8D800013EE8E72DE9F3411C4601219046089E08
:10B8E800099DFFF775FDC4F31302C4F30A54074614
:10B8F80034BB0192B8F1000F27D002A840F8088D98
:10B90800FFF70BFE0099F0B1019AC0F1200302FA8B
:10B9180003F30B43C2407B610192019B002B14BFD0
:10B9280002210121BB613961C4B1A4F2334404444A
:10B938003460C0F135002860384602B0BDE8F081B7
:10B9480042F48012D5E77961E7E701A8FFF7E5FD42
:10B958000121019B39617B612030E5E7A0F232408B
:10B9680007EB810330601869FFF7B8FDC0EB4110A1
:10B97800E1E738B502FB01F4214600F055F8054629
:10B9880018B122460021FDF764FE284638BD0000A4
:10B9980038B50546002943D051F8043C0C1F002B4C
:10B9A800B8BFE41800F098FA1E4A1368104633B975
:10B9B800636014602846BDE8384000F08EBAA342A0
:10B9C8000BD921686218934201BF1A685B68521844
:10B9D800226063600460EDE713465A680AB1A24228
:10B9E800FAD919685818A0420BD120680144581890
:10B9F80082421960DED110685268014419605A60A9
:10BA0800D8E702D90C232B60D4E7206821188A4292
:10BA180001BF116852680918216062605C60C9E75B
:10BA280038BD00BF5404002070B5CD1C25F00305B7
:10BA380008350C2D38BF0C25002D064601DBA94220
:10BA480003D90C233360002070BD00F045FA234A67
:10BA58001468214691B9224C23681BB9304600F07E
:10BA68007FF920602946304600F07AF9431C26D138
:10BA78000C233046336000F030FAE4E70B685B1BB8
:10BA88001AD40B2B0FD90B60CC18CD50304600F0D0
:10BA980024FA04F10B00231D20F00700C31A1BD061
:10BAA8005A42E25070BD8C420BBF63684B6813600A
:10BAB800636018BF0C46E9E70C464968CAE7C41C2E
:10BAC80024F00304A04205D0211A304600F048F9BA
:10BAD8000130CDD02560D9E770BD00BF54040020E7
:10BAE80058040020936810B4013B002B936008DAD7
:10BAF8009469A34202DBCBB20A2B02D110BCFEF739
:10BB080043BB1368581C10601970C8B210BC70474A
:10BB1800F8B506460F461446D518AC4201D10020A8
:10BB280007E03A4614F8011B3046FFF7DBFF431CD9
:10BB3800F3D1F8BD2DE9F04F9DB00C46174603939D
:10BB4800064618B183690BB9FFF730FB7C4B9C4262
:10BB580057D17468A38918075DD52369002B5AD07B
:10BB68000023099320238DF8293030234FF0010B4F
:10BB78008DF82A30B846454615F8013B002B55D1BB
:10BB8800B8EB070A0BD053463A4621463046FFF732
:10BB9800BFFF013000F0C480099B5344099398F813
:10BBA8000030002B00F0BC8000234FF0FF320493DC
:10BBB8000793059206938DF853301A930522297836
:10BBC8006048FFF7F7FB05F10108049B002831D115
:10BBD800D90644BF20228DF853201A0744BF2B22D0
:10BBE8008DF853202A782A2A2CD000210A20079A77
:10BBF800A84698F800300135303B092B6DD971B350
:10BC080026E0514B9C4201D1B468A3E74F4B9C42BC
:10BC180008BFF4689EE721463046FEF707FB002878
:10BC28009ED04FF0FF301DB0BDE8F08F252BA7D078
:10BC3800A846A0E7434A4546801A0BFA00F0184385
:10BC48000490BBE7039A111D12680391002A01DBD7
:10BC5800079204E0524243F002030792049398F8D3
:10BC680000302E2B10D198F8013008F101012A2B51
:10BC780037D1039B08F102081A1D1B680392002B99
:10BC8800B8BF4FF0FF330593314D032298F80010E9
:10BC98002846FFF78FFB40B14023401B03FA00F012
:10BCA800049B08F101080343049398F80010062246
:10BCB800284808F101078DF82810FFF77BFB0028BA
:10BCC80034D0254B03BB039B073323F0070308330A
:10BCD8000393099B4B4409934CE700FB0232012173
:10BCE80086E700230A2518460593884698F8002019
:10BCF8000131303A092A03D9002BC5D00590C3E792
:10BD080005FB00200123F0E703AB00932246134B09
:10BD180004A93046FDF736FDB0F1FF3F8146D8D182
:10BD2800A3895B063FF57DAF09987CE703AB0093D9
:10BD380022460A4B04A93046FDF7D4FFECE700BFC2
:10BD480068C00008A4C1000888C0000848C00008EE
:10BD5800AAC10008AEC100088D97000819BB0008E9
:10BD680038B50023054C054608462360FCF7BEFE9F
:10BD7800431C02D1236803B12B6038BD9C170020F7
:10BD880010B50C46B1F90E1000F0A8F80028ABBFAA
:10BD9800636DA3891B1823F48053ACBF6365A3812B
:10BDA80010BD2DE9F0411F468B890546DB050C4681
:10BDB800164605D502230022B1F90E1000F068F8E6
:10BDC800A389324623F48053A381B4F90E103B466D
:10BDD8002846BDE8F04100F017B810B50C46B1F997
:10BDE8000E1000F055F8431CA38915BF606523F4B5
:10BDF800805343F48053A38118BFA38110BDB1F9C8
:10BE08000E1000F013B8000038B505460846114674
:10BE18000022054C22601A46FBF7ACFF431C02D1F6
:10BE2800236803B12B6038BD9C17002038B5002368
:10BE3800054C054608462360FCF772FE431C02D1F8
:10BE4800236803B12B6038BD9C17002038B5002348
:10BE5800064C0546084611462360FCF764FE431C61
:10BE680002D1236803B12B6038BD00BF9C170020A6
:10BE780038B50023054C054608462360FCF758FEF4
:10BE8800431C02D1236803B12B6038BD9C170020E6
:10BE980038B50546084611460022054C22601A4668
:10BEA800FCF748FE431C02D1236803B12B6038BD60
:10BEB8009C17002082B001B901A942B14BB1137897
:10BEC8000B601278101C18BF012002B07047104692
:10BED800FBE76FF00100F8E77047704738B5054693
:10BEE800084611460022054C22601A46FCF7F0FD70
:10BEF800431C02D1236803B12B6038BD9C17002076
:10BF080049B1FF2A8BBF8A230A700360012088BFCA
:10BF18004FF0FF307047084670470000F8B500BF83
:10BF2800F8BC08BC9E467047F8B500BFF8BC08BC12
:04BF38009E4670476A
:10BF400002030405060708090A0B0C0D0E0F10105A
:10BF500002030405060708090A0B0C0D0E0F10104A
:10BF600000080140008000000010014000080000AF
:10BF70000010014040000000000801400080000067
:10BF80000010014000080000001001408000000087
:10BF9000457261736572204572726F720D0057723F
:10BFA000697465204572726F722025640D0A000065
:10BFB0000000000000000001020304060708090059
:10BFC000000000010203042530327820005265731E
:10BFD0006574205374617274200D00504F574552A0
:10BFE000203A202564200D0A00504C4C2043545226
:10BFF0004C205354415254202121200D00000000B8
:10C0000038020020494E4600696E66004E414E00DF
:10C010006E616E00300030313233343536373839A6
:10C0200041424344454600303132333435363738A7
:10C030003961626364656600496E66696E69747928
:10C04000004E614E000000000000000000000000F3
:10C0500000000000000000000000000000000000E0
:10C0600000000000000000000000000000000000D0
:10C0700000000000000000000000000000000000C0
:10C0800000000000000000000000000000000000B0
:10C0900000000000000000000000000000000000A0
:10C0A00000000000000000000080E03779C3414339
:10C0B000176E05B5B5B89346F5F93FE9034F384D0E
:10C0C000321D30F94877825A3CBF737FDD4F1575BA
:10C0D000000000000000F03F0000000000002440CD
:10C0E00000000000000059400000000000408F40A8
:10C0F000000000000088C34000000000006AF84013
:10C100000000000080842E4100000000D012634136
:10C110000000000084D797410000000065CDCD41AC
:10C12000000000205FA00242000000E8764837428D
:10C13000000000A2941A6D42000040E59C30A2422B
:10C140000000901EC4BCD64200003426F56B0C43A0
:10C150000080E03779C3414300A0D8855734764347
:10C1600000C84E676DC1AB43003D9160E458E143A8
:10C17000408CB5781DAF154450EFE2D6E41A4B441D
:10C1800092D54D06CFF08044F64AE1C7022DB54462
:10C19000B49DD9794378EA440500000019000000F5
:10C1A0007D000000232D302B2000686C4C0065665C
:10C1B00067454647004300504F534958002E000042
:10C1C0002020202020202020202828282828202047
:10C1D000202020202020202020202020202020205F
:10C1E00088101010101010101010101010101010D7
:10C1F00004040404040404040404101010101010B7
:10C20000104141414141410101010101010101018F
:10C2100001010101010101010101011010101010C3
:10C220001042424242424202020202020202020260
:10C230000202020202020202020202101010102088
:10C2400000000000000000000000000000000000EE
:10C2500000000000000000000000000000000000DE
:10C2600000000000000000000000000000000000CE
:10C2700000000000000000000000000000000000BE
:10C2800000000000000000000000000000000000AE
:10C29000000000000000000000000000000000009E
:10C2A000000000000000000000000000000000008E
:10C2B000000000000000000000000000000000007E
:08C2C000BC8EFF7F01000000AD
:04C2C8000D4200081B
:04C2CC00E94100083C
:10C2D00001000000100000000014014000080000F0
:10C2E0000014014000040000001801400400000098
:10C2F0000014014000080000001401400004000088
:10C30000001801400800000000140140000800006F
:10C31000001401400004000000180140100000005B
:10C320000014014000080000001401400004000057
:10C330000018014020000000001401400008000027
:10C34000001401400004000000180140100000002B
:10C350000014014000080000001401400004000027
:10C3600000100140002000000014014000080000FF
:10C370000014014000040000001C014010000000F7
:10C3800000140140000800000014014000040000F7
:10C39000001C0140200000000014014000080000C3
:10C3A0000014014000040000001C01404000000097
:10C3B00000140140000800000014014000040000C7
:10C3C000001C014080000000001401400008000033
:10C3D0000014014000040000001C014000010000A6
:10C3E0000014014000080000001401400004000097
:10C3F000001C014000020000001401400100000088
:10C400000014014010000000001401400200000070
:10C410000014014001000000001401402000000051
:10C42000001401400200000000140140010000005F
:10C430000014014040000000001401400200000010
:10C44000001401400100000000140140040000003D
:10C45000001401400200000000140140010000002F
:10C460000014014008000000001401400200000018
:10C47000001401400002000000140140000100000F
:10C48000001C0140010000000014014000020000F7
:10C490000014014000010000001C014002000000E7
:10C4A00000140140000200000014014000010000DF
:10C4B000000C0140080000000014014000020000D0
:10C4C0000014014000010000000C014010000000B9
:10C4D00000A24A0400080140008000000010014052
:10C4E000000800000010014080000000000801402A
:10C4F0000080000000100140000800000010014012
:10C5000040000000380200200000000068C0000861
:10C5100088C0000848C000080000000000000000BB
:10C52000000000000000000000000000000000000B
:10C5300000000000000000000000000000000000FB
:10C5400000000000000000000000000000000000EB
:10C5500000000000000000000000000000000000DB
:10C560000000000000000000430000000000000088
:10C5700000000000000000000000000000000000BB
:10C580000000000000000000430000000000000068
:10C59000000000000000000000000000000000009B
:10C5A0000000000000000000430000000000000048
:10C5B000000000000000000000000000000000007B
:10C5C0000000000000000000430000000000000028
:10C5D000000000000000000000000000000000005B
:10C5E0000000000000000000430000000000000008
:10C5F000000000000000000000000000000000003B
:10C6000000000000000000004300000000000000E7
:10C61000000000000000000000000000000000001A
:10C6200000000000000000004300000000000000C7
:10C6300000000000000000000000000000000000FA
:10C64000000000000000000009BF0008BDBE000897
:10C6500000000000BFC10008BDC10008E8BF00081D
:10C66000E8BF0008E8BF0008E8BF0008E8BF00080E
:10C67000E8BF0008E8BF0008E8BF0008E8BF0008FE
:10C68000FFFFFFFFFFFFFFFFFFFFFFFFFFFF0000B8
:10C690000100415343494900000000000000000030
:10C6A000000000000000000000000000000000008A
:10C6B0000000415343494900000000000000000011
:10C6C000000000000000000000000000000000006A
:04C6D0000000000066
:04000005080095A5B5
:00000001FF
